:020000040000FA
:04000000EDEF1BF015
:08000800056ED8CF06F0E0CF31
:1000100007F00001E9CF0DF0EACF08F0E1CF09F0D9
:10002000E2CF0AF0D9CF0BF0DACF0CF0F3CF14F017
:10003000F4CF15F0FACF16F000C00FF001C010F0A9
:1000400002C011F003C012F004C013F0F2AA2CEFAA
:1000500000F0F2B4D8EF04F09DA032EF00F09EB0B3
:10006000FEEF04F0F2A838EF00F0F2B2F2EF05F084
:100070009DAA3EEF00F09EBAE7EF05F00FC000F03A
:1000800010C001F011C002F012C003F013C004F060
:100090000E8E0DC0E9FF08C0EAFF09C0E1FF0AC0EB
:1000A000E2FF0BC0D9FF0CC0DAFF14C0F3FF15C08C
:1000B000F4FF16C0FAFF055007C0E0FF06C0D8FFE6
:1000C0001000F2CF0EF0F29EF76ADC0FF66E000E13
:1000D000F7220900F5500EBEF28E1200D04B896E49
:1000E000DAF7A517F8D8CC3B7623C11D539E5D39AE
:1000F000E0C203CFCD95CB1681AB0A8EFB63F9F43A
:10010000901011EE25C56F9704C068075F96436590
:10011000450F84BA579CCE1BA614B6A35CC677D5F0
:10012000B43D9827B9133A2D214018A028DEAC839E
:10013000E3DD696CB1B7492B9D0CC77109F57E826F
:100140006A78D2D71FA7F64C8BC3EF32E5A9377A6E
:10015000D41E7006558D52EC152059DBADBC7F4A7C
:10016000D6BBBEB03E7BBD79B894E12201C41C3140
:100170002E4F4D3675F0AFF28CE70D80196192E489
:10018000B3744635B212FE4E6D9BF1E951FF9FCA22
:100190006602AE0E93EA3C0854346264E691D37D65
:1001A0000BB5A41A5A86A12447DF8FE8883F443351
:1001B00060F34241EB2F9AEDFC48D1728A7356FAF4
:1001C000055E852A2C58E267FD7CA85B30D9385043
:1001D00087DC6BBFC9A29926AA29C800F2CF0EF00E
:1001E000F29EF76AF60FF66E010EF7220900F5503F
:1001F0000EBEF28E12004669726D776172652056EE
:10020000312E3220434320323030312D32303036DF
:10021000205261706861656C20416272616D732C5F
:10022000202E746575746869732E636F6D00F2CF4C
:100230000EF0F29EF76A480FF66E020EF7220900E2
:10024000F5500EBEF28E120070726F626C656D20FA
:10025000696E697469616C697A696E67206361723D
:10026000642C20676F696E6720746F20736C6565FE
:100270007000F2CF0EF0F29EF76A8C0FF66E020E4F
:10028000F7220900F5500EBEF28E120070726F62F6
:100290006C656D2072656164696E67204250420032
:1002A000F2CF0EF0F29EF76ABA0FF66E020EF72248
:1002B0000900F5500EBEF28E120066696C6520735F
:1002C000797374656D20666F756E6400F2CF0EF001
:1002D000F29EF76AE60FF66E020EF7220900F5505D
:1002E0000EBEF28E1200726F6F74206469722073FA
:1002F000697A6520697320257500F2CF0EF0F29EB1
:10030000F76A140FF66E030EF7220900F5500EBEC1
:10031000F28E1200535049207468726F74746C65C9
:100320003D2046415354212074686973206D6F64E9
:100330006520646F6573206E6F7420737570706FC5
:10034000727420616C6C2063617264732100F2CF5F
:100350000EF0F29EF76A680FF66E030EF7220900A0
:10036000F5500EBEF28E1200535049207468726F21
:1003700074746C653D20534C4F570000F2CF0EF063
:10038000F29EF76A960FF66E030EF7220900F550FB
:100390000EBEF28E12004D4F444520697320534526
:1003A0005249414C5F4E4F50494E0000F2CF0EF083
:1003B000F29EF76AC60FF66E030EF7220900F5509B
:1003C0000EBEF28E12004D4F4445206973205345F6
:1003D0005249414C5F46554C4C5F4E4F50494E0080
:1003E000F2CF0EF0F29EF76AFA0FF66E030EF722C6
:1003F0000900F5500EBEF28E12004D4F44452069A3
:10040000732053455249414C5F46554C4C00F2CF46
:100410000EF0F29EF76A280FF66E040EF72209001E
:10042000F5500EBEF28E12004D4F444520697320E8
:1004300050494E20544F20504C415900F2CF0EF0FD
:10044000F29EF76A560FF66E040EF7220900F55079
:100450000EBEF28E12004D4F444520697320464F68
:1004600055522D464F555200F2CF0EF0F29EF76ACC
:10047000820FF66E040EF7220900F5500EBEF28EC2
:1004800012004D4F444520697320504152414C4C5D
:10049000454C20504F525400F2CF0EF0F29EF76AB6
:1004A000B20FF66E040EF7220900F5500EBEF28E62
:1004B00012004D4F44452069732053485546464C21
:1004C000452F52414E444F4D0000F2CF0EF0F29EA8
:1004D000F76AE40FF66E040EF7220900F5500EBE1F
:1004E000F28E12004D4F4445206973204445464129
:1004F000554C5400F2CF0EF0F29EF76A0E0FF66ED6
:10050000050EF7220900F5500EBEF28E12006C6F38
:100510007374206120736563746F72210000F2CFE1
:100520000EF0F29EF76A380FF66E050EF7220900FC
:10053000F5500EBEF28E12005F736F6E67207374FB
:100540006F7070656420627920757365725F00005A
:10055000F2CF0EF0F29EF76A6A0FF66E050EF722E2
:100560000900F5500EBEF28E1200736F6D652069A2
:100570006E666F2061626F757420636172643A0009
:10058000F2CF0EF0F29EF76A9A0FF66E050EF72282
:100590000900F5500EBEF28E120020627062737474
:1005A0003A25344C58202000F2CF0EF0F29EF76A24
:1005B000C20FF66E050EF7220900F5500EBEF28E40
:1005C0001200204250425F62707365633A25344CDA
:1005D00058202000F2CF0EF0F29EF76AEE0FF66E72
:1005E000050EF7220900F5500EBEF28E12002042D1
:1005F00050425F53635065433A25344C58202000E5
:10060000F2CF0EF0F29EF76A1A0FF66E060EF72280
:100610000900F5500EBEF28E1200204250425F5289
:10062000737664536343743A25344C582020000099
:10063000F2CF0EF0F29EF76A4A0FF66E060EF72220
:100640000900F5500EBEF28E1200204250425F4E5D
:100650006D4641543A25344C58202000F2CF0EF01C
:10066000F29EF76A760FF66E060EF7220900F55035
:100670000EBEF28E12002066617473746172743A59
:100680002025344C58202000F2CF0EF0F29EF76A5D
:10069000A20FF66E060EF7220900F5500EBEF28E7E
:1006A0001200204669727374446174615365637407
:1006B0006F723A25344C58202000F2CF0EF0F29E93
:1006C000F76AD40FF66E060EF7220900F5500EBE3B
:1006D000F28E120070726F626C656D2072656164DB
:1006E000696E6720666174207461626C652C20718C
:1006F00075697474696E6720636861696E2E205332
:100700006F7272792100F2CF0EF0F29EF76A200F1D
:10071000F66E070EF7220900F5500EBEF28E12009B
:100720005653313031313A206861726420726573FA
:1007300065740000F2CF0EF0F29EF76A4E0FF66E6F
:10074000070EF7220900F5500EBEF28E1200200AA5
:100750000D00F2CF0EF0F29EF76A6C0FF66E070EE8
:10076000F7220900F5500EBEF28E12004D4D432FB8
:10077000534420696E69743A2053656E7420307852
:1007800034302028636D643029205350490A0D000D
:10079000F2CF0EF0F29EF76AAA0FF66E070EF7225E
:1007A0000900F5500EBEF28E12004D4D432F5344FA
:1007B00020696E69743A20476F7420726573706F98
:1007C0006E7365200A0D0000F2CF0EF0F29EF76AFC
:1007D000E20FF66E070EF7220900F5500EBEF28EFC
:1007E0001200534420696E69743A20636F6D6D6125
:1007F0006E6435350000F2CF0EF0F29EF76A100FEE
:10080000F66E080EF7220900F5500EBEF28E1200A9
:100810006E6F7420616E2053442C206D6179626587
:1008200020616E206D6D633F0000F2CF0EF0F29EEE
:10083000F76A440FF66E080EF7220900F5500EBE57
:10084000F28E12007965732C206974277320616E13
:10085000206D6D632100F2CF0EF0F29EF76A700FEB
:10086000F66E080EF7220900F5500EBEF28E120049
:100870006661696C6564206F7574206F66206964B9
:100880006C650000F2CF0EF0F29EF76A9E0FF66ED6
:10089000080EF7220900F5500EBEF28E12004D4DE3
:1008A000432F534420696E69743A20476F74206F58
:1008B0007574206F662069646C6520726573706F53
:1008C0006E7365200A0D0000F2CF0EF0F29EF76AFB
:1008D000E20FF66E080EF7220900F5500EBEF28EFA
:1008E00012004D4D432F534420696E69743A2047DE
:1008F0006F742073657420626C6F636B206C656E1F
:1009000067746820726573706F6E73652E20446F14
:100910006E652E0A0D00F2CF0EF0F29EF76A300FD0
:10092000F66E090EF7220900F5500EBEF28E120087
:100930004920616D20746865204B696E6720000056
:10094000F2CF0EF0F29EF76A5A0FF66E090EF722FA
:100950000900F5500EBEF28E12006F6620467261DD
:100960006E6365210000F2CF0EF0F29EF76A800FF1
:10097000F66E090EF7220900F5500EBEF28E120037
:1009800077686F2061746500F2CF0EF0F29EF76A0F
:10099000A20FF66E090EF7220900F5500EBEF28E78
:1009A0001200616C6C20746865207069653F2100DD
:1009B000DE5312E183B408D0DB3D01D001D0DB2B44
:1009C000DC3D01D001D0DC2B83B606D0DB5301E047
:1009D000DB07DC5301E0DC07DA2D06D083CFDBF048
:1009E000F00EDB17DBC0DCF0DA51050804E183CF41
:1009F000DBF083CFDCF0F2943EEF00F09E903EEF10
:100A000000F0F29CF29EF2BEFDD79D9A9EAAFED700
:100A1000AECFEDF30301ED519EA8FED7AD6EED51C3
:100A2000BF080BE2C00EED5FED51040DF3CFEDF307
:100A3000EDC3DBF0EDC3DCF01DD0ED51B80804E1EF
:100A40000001E07D16D00301ED51B70804E100017B
:100A5000E0990FD00301ED51B60804E10001E089EF
:100A600008D00301ED51B50805E10001E081E093F4
:100A7000E09D0301ED51B40807E30001E081E0834C
:100A8000E09D300EDD6F0301C00EF2129D8A000161
:100A9000EBEF05F0F29CF29EF2BEFDD79D9A9EAA66
:100AA000FED7AECFEDF30301ED519EA8FED7AD6E9C
:100AB0000001DD516C0805E1EDC3DBF0300EDD6FA8
:100AC00080D0DD51720805E1EDC3DCF0300EDD6F42
:100AD00078D0DD51760807E1EDC3DCF0EDC3DBF043
:100AE000300EDD6F6ED0DD513008D8A46AD003011E
:100AF000ED516C0805E16C0E0001DD6F62D0030161
:100B0000ED51720805E1720E0001DD6F5AD003014C
:100B1000ED51760805E1760E0001DD6F52D003013C
:100B2000ED51610806E10001E099300EDD6F49D01A
:100B30000301ED51620806E10001E089300EDD6F2E
:100B400040D00301ED516B0808E10001E081E09322
:100B5000300EDD6FE09D35D00301ED5174082CE1BE
:100B60009EAAFED7AECFEDF3ED519EA8FED7AD6E97
:100B7000EF6BEDC3EEF3EEC3EFF3EE6B9EAAFED781
:100B8000AECFEDF3ED519EA8FED7AD6EED51EE2741
:100B9000000EEF23EFC3F1F3EEC3F0F30001E081A9
:100BA000E083F56BF46BF1C3F3F0F0C3F2F0E09D7A
:100BB000300EDD6F06D00301ED51700803E1000136
:100BC000E07D0301C00EF2129D8A0001000CDA5193
:100BD000030801E116D7DA51060801E15BDF9E9AAE
:100BE0003EEF00F0DA51020804E1F29853DFF2928E
:100BF000F288DA51040818E184A00CD0740E9EA883
:100C0000FED7AD6EF56BF46BF36B83CFF2F0E08142
:100C1000E083E08784B008D0760E9EA8FED7AD6E44
:100C200083CFDBF0DBC0DCF0DA2D11D083509EA83F
:100C3000FED7AD6EF56BF46BF36B83CFF2F00F0E56
:100C4000F217F36BF46BF56BE081E083E087DA5128
:100C5000050801E1E081F2923EEF00F0030EEA6E3A
:100C6000E10EE96EEF500EE00C0E016E006A002EF0
:100C7000FED7012EFBD7F70E006E002EFED700D058
:100C8000EF2EF2D7000C03016D532EE1040E6E6FB0
:100C9000C80EE16F0001E2DF03016E2FF9D76E6B22
:100CA0006E51000138DE03016E2B006E00509EA8CD
:100CB000FED7AD6E0E0E6E5DF3E16E6B6E510001F0
:100CC0003FDE03016E2B006E00509EA8FED7AD6E76
:100CD0000A0E6E5DF3E1020E6E6FC80EE16F000149
:100CE000BDDF03016E2FF9D76D2D46D0040E6E6F58
:100CF000C80EE16F0001B2DF03016E2FF9D7FE0EBF
:100D00009EA8FED7AD6E010E9EA8FED7AD6EFE0E5C
:100D10009EA8FED7AD6E020E9EA8FED7AD6E6E6B7E
:100D20006E51000120DE03016E2B006E00509EA864
:100D3000FED7AD6E070E6E5DF3E1FE0E9EA8FED7E8
:100D4000AD6EC00E9EA8FED7AD6E6E6B6E510001EB
:100D50001BDE03016E2B006E00509EA8FED7AD6E09
:100D60000D0E6E5DF3E1020E6E6FC80EE16F0001B5
:100D700075DF03016E2FF9D7000152EF1CF0020E50
:100D800003016D5F0CE3030EEA6E6D0EE96EEF502A
:100D900006E0020E006E002EFED7EF2EFAD70001FD
:100DA000AAEF1CF00301986B070E996F8B96030E48
:100DB000006E002EFED797C300F09951016E04E03B
:100DC000D8900032012EFCD78B9800B08B888B8690
:100DD000210E006E002EFED782A00BD0010E006EF9
:100DE0009951016E04E0D8900036012EFCD70050D6
:100DF00098138B96210E006E002EFED799519907FD
:100E0000000AD9E198C301F00001000CC66A8B8288
:100E10008A8694988A9894968DC397F3C3DF8EC37D
:100E200097F3C0DF030E0301946F910E936F010ED1
:100E30009325016E000E9421036E01C095F3966F09
:100E40008FC397F30001AEDF96C3EAFF95C3E9FFB6
:100E500001C0EFFF030E0301946F910E936F94C3D3
:100E600003F0956F94C396F390C397F300019ADF54
:100E700096C3EAFF95C3E9FF01C0EFFF8A88948813
:100E80005FC3C6FF030191C301F092C302F00001EA
:100E9000000C0301E551016AE45D03E2E4C300F0E4
:100EA0000CD0006A080EE66FE4370036E551005CAE
:100EB000D8B0006E0136E62FF7D70001000C0150C4
:100EC000E2C3E4F3640E0301E56F0001E2DF00C05A
:100ED000E2F30150300E08E10301E3A30ED0E3B7C3
:100EE0000CD0E3B9200E04D00301E397E399E3812A
:100EF000012601509EA8FED7AD6EE2C3E4F30A0EB0
:100F0000E56F0001C6DF00C0E2F30150300E08E1DA
:100F10000301E3B70BD0E3A109D0E3B9200E000130
:100F2000012601509EA8FED7AD6E0301300EE227C8
:100F3000E2519EA8FED7AD6E0001000C0301E06BEC
:100F4000E0510908D8A0F2D28B808B961E0EE16F7B
:100F5000000184DEC78C220EC66E8B828B901E0E23
:100F60000301E16F00017ADE0301DE6BDE51090847
:100F700007E3C950FF0EC96EC7A0FED7DE2BF6D718
:100F80008B92C950400EC96EC7A0FED7C950C96A1E
:100F9000C7A0FED7C950C96AC7A0FED7C950C96A41
:100FA000C7A0FED7C950C96AC7A0FED7C950950EC1
:100FB000C96EC7A0FED7DD532EE0E16BE151000101
:100FC0009AEC03F0000907E00301E12B9EA8FED78D
:100FD000AD6EF4D700010D0E9EA8FED7AD6E0A0EC1
:100FE0009EA8FED7AD6E0301E16BE1510001A9ECB3
:100FF00003F0000907E00301E12B9EA8FED7AD6EC8
:10100000F4D700010D0E9EA8FED7AD6E0A0E9EA865
:10101000FED7AD6E0301010EE76F020EE96F080EF9
:10102000E86FE85302E1E95312E0C950FF0EC96EC0
:10103000C7A0FED7C9CFEAF3E751EA5D03E1000E8E
:10104000016E07D0E851D8B4E907E807EAD7010EE6
:10105000016E0152D8A468D2DD5317E0E16BE15173
:101060000001C8EC03F0000907E00301E12B9EA892
:10107000FED7AD6EF4D700010D0E9EA8FED7AD6E63
:101080000A0E9EA8FED7AD6E0301DE6BDF6BDD534B
:1010900027E00D0E9EA8FED7AD6E0A0E9EA8FED7C5
:1010A000AD6EE16BE1510001E4EC03F00301E12BD3
:1010B000006E00509EA8FED7AD6E120EE15DF2E10B
:1010C000030EE26F2E0E9EA8FED7AD6EE22FFAD76A
:1010D0000D0E9EA8FED7AD6E0A0E9EA8FED7AD6E71
:1010E0008B82C950FF0EC96EC7A0FED7C950FF0E34
:1010F000C96EC7A0FED78B92C950770EC96EC7A024
:10110000FED7C950C96AC7A0FED7C950C96AC7A0CF
:10111000FED7C950C96AC7A0FED7C950C96AC7A0BF
:10112000FED7C950F00EC96EC7A0FED7800EE16F82
:10113000020EE36F080EE26FE25302E1E35313E0A5
:10114000C950FF0EC96EC7A0FED7C9CFE4F3E15165
:10115000E417E45303E1000E016E07D0E251D8B466
:10116000E307E207E9D7010E016E012C91D0DE2BD7
:10117000DE510A08D8B08BD0DF6BDD5317E0E16B8E
:10118000E1510001FBEC03F00301E12B006E005084
:101190009EA8FED7AD6E180EE15DF2E10D0E9EA881
:1011A000FED7AD6E0A0E9EA8FED7AD6E8B82C950DB
:1011B000FF0EC96EC7A0FED7C950FF0EC96EC7A0EB
:1011C000FED78B92C950410EC96EC7A0FED7C95039
:1011D000C96AC7A0FED7C950C96AC7A0FED7C950FF
:1011E000C96AC7A0FED7C950C96AC7A0FED7C950EF
:1011F000FF0EC96EC7A0FED7DF2BDD530BE02E0E0E
:101200009EA8FED7AD6EDFC3E2F31B0EE36F0001B5
:1012100056DE0301810EE16F020EE36F080EE26FEE
:10122000E25302E1E35313E0C950FF0EC96EC7A0B9
:10123000FED7C9CFE4F3E151E417E45303E1000E14
:10124000016E07D0E251D8B4E307E207E9D7010EF7
:10125000016E01521AE1DD5317E0E16BE15100012B
:1012600015EC04F00301E12B006E00509EA8FED7A0
:10127000AD6E110EE15DF2E10D0E9EA8FED7AD6ED2
:101280000A0E9EA8FED7AD6E93D0DF3D8FD74ED706
:10129000C950FF0EC96EC7A0FED7C950FF0EC96E58
:1012A000C7A0FED7C950FF0EC96EC7A0FED7C95050
:1012B000FF0EC96EC7A0FED7C950690EC96EC7A080
:1012C000FED7C950C96AC7A0FED7C950C96AC7A00E
:1012D000FED7C950C96AC7A0FED7C950C96AC7A0FE
:1012E000FED7C950FF0EC96EC7A0FED7DE2BDD5357
:1012F00017E0030EE16F2E0E9EA8FED7AD6EE12F14
:10130000FAD7DEC3E2F31B0EE36F0001D8DD640EF3
:101310009EA8FED7AD6E200E9EA8FED7AD6E03012F
:10132000810EE16F020EE36F080EE26FE25302E1FD
:10133000E35313E0C950FF0EC96EC7A0FED7C9CF53
:10134000E4F3E151E417E45303E1000E016E07D02A
:10135000E251D8B4E307E207E9D7010E016E01526A
:1013600001E126D0DE3D93D6DD531FE0E16BE15174
:1013700000012BEC04F00301E12B006E00509EA84D
:10138000FED7AD6E120EE15DF2E1030EE26F2D0E9F
:101390009EA8FED7AD6EE22FFAD70D0E9EA8FED7FF
:1013A000AD6E0A0E9EA8FED7AD6E010E016EBED0C8
:1013B000DD5327E00D0E9EA8FED7AD6E0A0E9EA847
:1013C000FED7AD6EE16BE151000142EC04F0000983
:1013D00007E00301E12B9EA8FED7AD6EF4D7000114
:1013E0000D0E9EA8FED7AD6E0A0E9EA8FED7AD6E5E
:1013F0000D0E9EA8FED7AD6E0A0E9EA8FED7AD6E4E
:1014000003018B82C950FF0EC96EC7A0FED7C95019
:10141000FF0EC96EC7A0FED7C950FF0EC96EC7A088
:10142000FED7C950FF0EC96EC7A0FED78B92C95018
:10143000FF0EC96EC7A0FED7C950500EC96EC7A017
:10144000FED7C950C96AC7A0FED7C950C96AC7A08C
:10145000FED7C950020EC96EC7A0FED7C950C96ACF
:10146000C7A0FED7C950FF0EC96EC7A0FED7E76B55
:10147000020EE96F080EE86FE85302E1E95312E04B
:10148000C950FF0EC96EC7A0FED7C9CFEAF3E75116
:10149000EA5D03E1000E016E07D0E851D8B4E90718
:1014A000E807EAD7010E016E012C03D0010E016E90
:1014B0003DD0C950FF0EC96EC7A0FED7C950FF0E60
:1014C000C96EC7A0FED78B82DD531FE0E16BE151EF
:1014D000000164EC04F0000907E00301E12B9EA881
:1014E000FED7AD6EF4D700010D0E9EA8FED7AD6EEF
:1014F0000A0E9EA8FED7AD6E0D0E9EA8FED7AD6E4D
:101500000A0E9EA8FED7AD6E0301C950FF0EC96E2C
:10151000C7A0FED7C950FF0EC96EC7A0FED75FC3D4
:10152000C6FF000E016E02D0E02B0AD50001000CB0
:101530000301E16BE1510908D8A0BED05FC3C6FF2B
:10154000D890E36BDD35E46FDE35E56FDF35E66FB0
:10155000C950FF0EC96EC7A0FED7C950FF0EC96E95
:10156000C7A0FED78B92C950510EC96EC7A0FED737
:10157000030EE86FE30EE76F030EE725016E000E22
:10158000E821036E01C0E9FFEA6EEFCFE9F3C9502D
:10159000E9C3C9FFC7A0FED7030EE86FE30EE76FEC
:1015A000020EE725016E000EE821036E01C0E9FF7F
:1015B000EA6EEFCFE9F3C950E9C3C9FFC7A0FED770
:1015C000030EE86FE30EE76F010EE725016E000ED4
:1015D000E821036E01C0E9FFEA6EEFCFE9F3C950DD
:1015E000E9C3C9FFC7A0FED7C950C96AC7A0FED7C3
:1015F000C950FF0EC96EC7A0FED7E76B020EE96F98
:10160000080EE86FE85302E1E95312E0C950FF0EFB
:10161000C96EC7A0FED7C9CFEAF3E751EA5D03E17F
:10162000000E016E07D0E851D8B4E907E807EAD701
:10163000010E016E015233E1FE0EE76F020EE96FFB
:10164000080EE86FE85302E1E95312E0C950FF0EBB
:10165000C96EC7A0FED7C9CFEAF3E751EA5D03E13F
:10166000000E016E07D0E851D8B4E907E807EAD7C1
:10167000010E016E015203E1000E016E1FD0E26BFC
:10168000E23D01D00CD0C950FF0EC96EC7A0FED7F5
:10169000C950FF0EC96EC7A0FED7E22BF1D78B82CF
:1016A000C950FF0EC96EC7A0FED7C950FF0EC96E44
:1016B000C7A0FED7E12B3ED7010E016E0001000C42
:1016C0000301DE530CE0C950FF0EC96EC7A0FED760
:1016D000C950FF0EC96EC7A0FED7DE07F2D70001C2
:1016E000000CC950FF0EC96EC7A0FED7C9CF18F0B5
:1016F000C950FF0EC96EC7A0FED7C9CF19F0000CA4
:10170000C950FF0EC96EC7A0FED7C950FF0EC96EE3
:10171000C7A0FED78B82C950FF0EC96EC7A0FED7E7
:10172000C950FF0EC96EC7A0FED7000C0301E76BBE
:10173000E86B010EE96FDA6AD96A030EEC6FDF0E0F
:10174000EB6F030EEA6EE30EE96EECC3E2FFEBC350
:10175000E1FFE9C3EAF3D890E550EE02F350E72346
:10176000F450E823EA2FF7D7E7C3DEFFE8C3E7F337
:10177000E86BD8B0E82BEB2BD8B4EC2BE92BE95174
:101780000508DFE10001000C030174BF10D00F0E4B
:10179000006E733900160A0E005C03E2300E00265C
:1017A00002D07451002600509EA8FED7AD6E0F0ED9
:1017B00073170A0E735D02E2300E02D0749F7451EB
:1017C000732773519EA8FED7AD6E0001000CE36B2A
:1017D000E26B0301E06BDF6BDE6BDD6B0001A8DE0B
:1017E000E30E0301DE6F00016BDF7BDF19C0E3F066
:1017F0000001E26B1850E227000EE3231B0E0301E9
:10180000DE6F00015DDF7CDF0301746B736BE3C08F
:1018100072F3E2C071F374C3E0F373C3DFF3E3C0A8
:10182000DEF3E2C0DDF3000183DE050E0301DE6FAF
:10183000000146DF56DFE96B19C0E8F052DF000E09
:101840000001E8271850E92319C0E1F04ADF03013D
:10185000736B185073250001E66F000E0301192009
:101860000001E76F3EDF18C01AF13BDF3ADF39DFD6
:10187000060E0301DE6F000123DF33DF0101156B6C
:10188000146B136B126B0301736B726B73C303F0F6
:1018900072C302F0006A005018240101126F000E9A
:1018A0001920136F000E0220146F000E0320156F15
:1018B00015C170F314C16FF313C16EF312C16DF350
:1018C00000010FDF0301736B726B73C303F072C30C
:1018D00002F0006A005018240101126F000E192056
:1018E000136F000E0220146F000E0320156F13C13A
:1018F00015F112C114F1126B136B03016D5101014B
:10190000122703016E510101132303016F510101DD
:10191000142303017051010115230001E2DEE1DE11
:10192000E0DE0301736B726B73C303F072C302F0EA
:10193000006A005018240101166F000E1920176F5D
:10194000000E0220186F000E0320196F19C170F3EA
:1019500018C16FF317C16EF316C16DF30001C1DE3C
:10196000E70E0301DE6F0001ABDECADE0301736B1D
:10197000726B73C303F072C302F0006A0050182444
:101980000101166F000E1920176F000E0220186F4C
:10199000000E0320196F17C119F116C118F1166B4B
:1019A000176B03016D510101162703016E510101EF
:1019B000172303016F510101182303017051010125
:1019C000192319C109F118C108F117C107F116C18E
:1019D00006F10001E651E225F66FE751E321F76FCA
:1019E000F86BF96B0301E26BE16BE06B1AC1DFF39B
:1019F00015C1E6F314C1E5F313C1E4F312C1E3F337
:101A0000000194DE0050E625E46F0150E721E56F08
:101A10000301746B736BE3C072F3E2C071F3E4C053
:101A200000F0026A036A005071250001FA6FE55167
:101A3000030172210001FB6F0250030173210001B9
:101A4000FC6F0350030174210001FD6F0D0E9EA871
:101A5000FED7AD6E0A0E9EA8FED7AD6E0301716B68
:101A600071510001A8EC02F00301712B006E0050CF
:101A70009EA8FED7AD6E150E715DF2E10D0E9EA80B
:101A8000FED7AD6E0A0E9EA8FED7AD6E716B71517A
:101A90000001C0EC02F00301712B006E00509EA803
:101AA000FED7AD6E070E715DF2E1E3C073F3370E42
:101AB000746F000169DEE2C073F3370E0301746FC7
:101AC000000162DE200E9EA8FED7AD6E200E9EA8FD
:101AD000FED7AD6E0D0E9EA8FED7AD6E0A0E9EA867
:101AE000FED7AD6E0301716B71510001D4EC02F0B1
:101AF0000301712B006E00509EA8FED7AD6E0B0E39
:101B0000715DF2E1E9C073F3370E746F00013CDEE2
:101B1000E8C073F3370E0301746F000135DE200E49
:101B20009EA8FED7AD6E200E9EA8FED7AD6E0D0E00
:101B30009EA8FED7AD6E0A0E9EA8FED7AD6E03011D
:101B4000716B71510001EAEC02F00301712B006E20
:101B500000509EA8FED7AD6E0B0E715DF2E1020E35
:101B6000726F300E9EA8FED7AD6E722FFAD7E1C00D
:101B700073F3370E746F000107DE200E9EA8FED7A8
:101B8000AD6E200E9EA8FED7AD6E0D0E9EA8FED7A0
:101B9000AD6E0A0E9EA8FED7AD6E0301716B71513A
:101BA000000100EC03F00301712B006E00509EA8B1
:101BB000FED7AD6E0E0E715DF2E1E7C073F3370E26
:101BC000746F0001E1DDE6C073F3370E0301746F3B
:101BD0000001DADD200E9EA8FED7AD6E200E9EA875
:101BE000FED7AD6E0D0E9EA8FED7AD6E0A0E9EA856
:101BF000FED7AD6E0301716B7151000118EC03F05B
:101C00000301712B006E00509EA8FED7AD6E0B0E27
:101C1000715DF2E1020E726F300E9EA8FED7AD6EBE
:101C2000722FFAD71AC173F3370E746F0001ACDD4F
:101C3000200E9EA8FED7AD6E200E9EA8FED7AD6EDC
:101C40000D0E9EA8FED7AD6E0A0E9EA8FED7AD6EF5
:101C50000301716B715100012EEC03F00301712B34
:101C6000006E00509EA8FED7AD6E0B0E715DF2E1C6
:101C7000F7C073F3370E746F000186DDF6C073F39F
:101C8000370E0301746F00017FDD200E9EA8FED782
:101C9000AD6E200E9EA8FED7AD6E0D0E9EA8FED78F
:101CA000AD6E0A0E9EA8FED7AD6E0301716B715129
:101CB000000144EC03F00301712B006E00509EA85C
:101CC000FED7AD6E110E715DF2E1E5C073F3370E14
:101CD000746F000159DDE4C073F3370E0301746FB4
:101CE000000152DD200E9EA8FED7AD6E200E9EA8EC
:101CF000FED7AD6E0D0E9EA8FED7AD6E0A0E9EA845
:101D0000FED7AD6E000C0301D76BD66BD890D237DF
:101D1000D337D437D537030EDE6FD20EE96EDEC36C
:101D2000EAFFEFCFDCF3D3C3D2F3D4C3D3F3D5C3ED
:101D3000D4F3D56B0001F6510301D2270001F7510E
:101D40000301D3230001F8510301D4230001F95109
:101D50000301D523D5C3E0F3D4C3DFF3D3C3DEF34C
:101D6000D2C3DDF3000198EC0AF0012C52D05E0ED4
:101D70009EA8FED7AD6ED5C3E0F3D4C3DFF3D3C3C3
:101D8000DEF3D2C3DDF398EC0AF0012C42D0260E2C
:101D90009EA8FED7AD6E0301DD6B00019EEC07F03F
:101DA000D5C3E0F3D4C3DFF3D3C3DEF3D2C3DDF393
:101DB00098EC0AF0012C2DD02A0E9EA8FED7AD6E0D
:101DC0000301DD6B00019EEC07F0D5C3E0F3D4C343
:101DD000DFF3D3C3DEF3D2C3DDF398EC0AF0012CBA
:101DE00018D00301DD6BDD5100015DEC03F0030150
:101DF000DD2B006E00509EA8FED7AD6E310EDD5D6E
:101E0000F2E1FF0E006E016E026E036E43D0000120
:101E1000E081DCC3DEF354DC64DC0301DF6B036AC6
:101E20001850DF25D66F03501920D76F000159DCF9
:101E30000301DB6BDA6BD96BD86BDF6B036A18506D
:101E4000DF25D86F03501920D96FDA6BDB6BD9C34C
:101E5000DBF3D8C3DAF3D86BD96B026A036AD651C5
:101E6000D827D751D9230250DA230350DB23FF0EA2
:101E7000D880DC55DD6FDE6F000122DC32DC31DC26
:101E80003FDCD8C300F0D9C301F0DAC302F0DBC3F2
:101E900003F003010001000C19C109F118C108F198
:101EA00017C107F116C106F10301706B6F6B6E6B02
:101EB0006D6B09C10DF108C10CF107C10BF106C131
:101EC0000AF10DC1D5F30CC1D4F30BC1D3F30AC190
:101ED000D2F3000118DF03C009F102C008F101C00C
:101EE00007F100C006F106C171F307C172F308C122
:101EF00073F3010109510F0B0301746F010E6D277C
:101F0000D8B06E2BD8B46F2BD8B4702B74510F0887
:101F10000CE3CFE17351FF0808E3CBE17251FF08F6
:101F200004E3C7E17151EE08C4E270C3E2F36FC38A
:101F3000E1F36EC3E0F36DC3DFF3E66BE56BE46BD7
:101F4000E1C0E3F3000196EC0BF003C011F102C015
:101F500010F101C00FF100C00EF101010E370F3773
:101F6000103711370E370F37103711370E370F373D
:101F7000103711370E370F3710371137F00E0E1795
:101F8000FF0E0E27D8A00F27D8A01027D8A0112702
:101F900000019EEF1DF0016A026A006A036A0301F4
:101FA000D55102E1D45118E0100ED66FD890D23737
:101FB000D33700360336D551035C02E1D451005CBF
:101FC00007E3D451005ED8A00306D551035ED88044
:101FD00001360236D62FEAD70001000C006A016AEA
:101FE000026A036A0301A86BA96BAA6BAB6BA751CA
:101FF000A611A511A4112CE0200EAC6FD890A0372B
:10200000A137A237A337A837A937AA37AB37A751CB
:10201000AB5D08E1A651AA5D05E1A551A95D02E10C
:10202000A451A85D0FE3A451A85FA551D8A0A53D78
:10203000A95FA651D8A0A63DAA5FA751D8A0A73DE9
:10204000AB5FD8800036013602360336AC2FD6D7C8
:10205000030EEA6EA80EE96E0001000C0301D251D6
:10206000D403F3CF01F0F4CF00F0D503F3500026F2
:10207000D351D403F3500020026E000181EF10F021
:102080000301D16BCA6BC96BC86BC76B19C109F16E
:1020900018C108F117C107F116C106F17431036EBA
:1020A0007331026E7231016E7131006E0332023291
:1020B0000132003203320232013200320332023284
:1020C0000132003200C0CDF301C0CEF3CEC3D0F355
:1020D000CDC3CFF3CEC3D3F3CDC3D2F3D56BE1C021
:1020E000D4F3000158DF02C0CEF301C0CDF3CEC35C
:1020F000D3F3CDC3D2F30301D56BE1C0D4F3000118
:10210000ADD702C0CCF301C0CBF30301CB51CF5DFF
:10211000CB6FCC51D059CC6FCD5302E1CE532AE0D6
:1021200009C10DF108C10CF107C10BF106C10AF19B
:102130000DC1D5F30CC1D4F30BC1D3F30AC1D2F353
:102140000001E1DD03C009F102C008F101C007F19F
:1021500000C006F106C1C7F307C1C8F308C1C9F33F
:10216000010109510F0B0301CA6FCD51D8B4CE073D
:10217000CD07D2D7CA510E0813E2FF0A0DE1C951AB
:10218000FE080EE2FF0A08E1C851FE0809E2FF0A54
:1021900003E1C751EF0804E2020E016ECFEF14F025
:1021A000020E0101065D0301C36F000E0101075914
:1021B0000301C46F000E010108590301C56F000E31
:1021C000010109590301C66FE1C000F0016A026A0A
:1021D000036A03C0D5F302C0D4F301C0D3F3E1C056
:1021E000D2F3C6C3E2F3C5C3E1F3C4C3E0F3C3C390
:1021F000DFF303C0E6F302C0E5F301C0E4F3E1C09E
:10220000E3F3000196EC0BF003C0C6F302C0C5F384
:1022100001C0C4F300C0C3F3FA510301C327000196
:10222000FB510301C4230001FC510301C52300013C
:10223000FD510301C623026A036ACB51C327CC5167
:10224000C4230250C5230350C623C6C3E0F3C5C34D
:10225000DFF3C4C3DEF3C3C3DDF3000198EC0AF07F
:10226000030171510F0BD26FD36BD46BD56BD23589
:10227000006ED335016ED435026ED535036E00364F
:102280000136023603360036013602360336003692
:10229000013602360336F00E001600C0D1F3D1C36A
:1022A000DEF3000160EC0BF00301B86BB8511F08BE
:1022B000D8A000D1000171EC0BF00301D12B036A0F
:1022C000B851BA0F016E000E032203C0D3F3036AA4
:1022D000B8519A0FE96E000E0320EA6EEFCFD4F3E7
:1022E000D3C3EAFF01C0E9FFD4C3EFFF036AB851CB
:1022F0009A0F016E000E032203C0D3F3036AB85194
:102300007A0FE96E000E0320EA6EEFCFD4F3D3C349
:10231000EAFF01C0E9FFD4C3EFFF036AB8517A0FA7
:10232000016E000E032203C0D3F3036AB8515A0FA3
:10233000E96E000E0320EA6EEFCFD4F3D3C3EAFFB9
:1023400001C0E9FFD4C3EFFF036AB8515A0F016E11
:10235000000E032203C0D3F3036AB8513A0FE96EAB
:10236000000E0320EA6EEFCFD4F3D3C3EAFF01C01F
:10237000E9FFD4C3EFFF036AB8513A0F016E000EB4
:10238000032203C0D3F3036AB8511A0FE96E000E9B
:102390000320EA6EEFCFD4F3D3C3EAFF01C0E9FF15
:1023A000D4C3EFFF036AB8511A0FE96E000E032081
:1023B000EA6E18C0EFFFB82B036AB851BA0F016E6E
:1023C000000E032203C0D3F3036AB8519A0FE96EDB
:1023D000000E0320EA6EEFCFD4F3D3C3EAFF01C0AF
:1023E000E9FFD4C3EFFF036AB8519A0F016E000EE4
:1023F000032203C0D3F3036AB8517A0FE96E000ECB
:102400000320EA6EEFCFD4F3D3C3EAFF01C0E9FFA4
:10241000D4C3EFFF036AB8517A0F016E000E032296
:1024200003C0D3F3036AB8515A0FE96E000E0320BC
:10243000EA6EEFCFD4F3D3C3EAFF01C0E9FFD4C300
:10244000EFFF036AB8515A0F016E000E032203C05A
:10245000D3F3036AB8513A0FE96E000E0320EA6E17
:10246000EFCFD4F3D3C3EAFF01C0E9FFD4C3EFFF3A
:10247000036AB8513A0F016E000E032203C0D3F372
:10248000036AB8511A0FE96E000E0320EA6EEFCF0F
:10249000D4F3D3C3EAFF01C0E9FFD4C3EFFF036A5B
:1024A000B8511A0FE96E000E0320EA6E19C0EFFF53
:1024B000B82BFCD6FF0ED880D155D26FDE6F00014D
:1024C00060EC0BF071EC0BF071EC0BF080EC0BF0AE
:1024D0001A52D8B44FD11A50E508D8B44BD10301E1
:1024E000B76BB96BB95114080BE3036AB951760F96
:1024F000E96E030E0320EA6EFF0EEF6EB92BF2D7E2
:10250000B86BB8C3B7F3B8510A081AE3B751010B57
:10251000006ED36BE8B0D38FB751FE0B006ED8902E
:1025200000320050D311D56F036AB8511A0FE96E0B
:10253000000E0320EA6EEF50D525B76FB82BE3D716
:10254000BB6B4750B75DD8A4FAD03BC076F33DC013
:1025500077F33FC078F341C079F343C07AF348C0C2
:102560007BF34AC07CF34CC07DF34EC07EF350C079
:102570007FF352C080F356C081F358C082F30D0E32
:10258000BB6FB96BB9510C080DE3036AB951760FF3
:10259000E96E030E0320EA6EEF5202E1B9C3BBF30A
:1025A000B92BF0D76750B75DD8A4C8D05BC083F310
:1025B0005DC084F35FC085F361C086F363C087F3B9
:1025C00068C088F36AC089F36CC08AF36EC08BF36D
:1025D00070C08CF372C08DF376C08EF378C08FF329
:1025E000190EBB6F0D0EB96FB95119080DE3036ACF
:1025F000B951760FE96E030E0320EA6EEF5202E145
:10260000B9C3BBF3B92BF0D7000187510301B75D04
:10261000D8A494D07BC090F37DC091F37FC092F397
:1026200081C093F383C094F388C095F38AC096F376
:102630008CC097F38EC098F390C099F392C09AF330
:1026400096C09BF398C09CF3260EBB6F1A0EB96F11
:10265000B95126080DE3036AB951760FE96E030EEE
:102660000320EA6EEF5202E1B9C3BBF3B92BF0D7F6
:102670000001A7510301B75D2EE19BC09DF39DC0F2
:102680009EF39FC09FF3A1C0A0F3A3C0A1F3A8C075
:10269000A2F3AAC0A3F3ACC0A4F3AEC0A5F3B0C02C
:1026A000A6F3B2C0A7F3B6C0A8F3B8C0A9F3330E1F
:1026B000BB6F270EB96FB95133080DE3036AB951E7
:1026C000760FE96E030E0320EA6EEF5202E1B9C302
:1026D000BBF3B92BF0D70001C7510301B75D2EE161
:1026E000BBC0AAF3BDC0ABF3BFC0ACF3C1C0ADF378
:1026F000C3C0AEF3C8C0AFF3CAC0B0F3CCC0B1F32F
:10270000CEC0B2F3D0C0B3F3D2C0B4F3D6C0B5F3E9
:10271000D8C0B6F3400EBB6F340EB96FB951400844
:102720000DE3036AB951760FE96E030E0320EA6EDA
:10273000EF5202E1B9C3BBF3B92BF0D71AD01AC0DC
:1027400076F31BC077F31CC078F31DC079F31EC06D
:102750007AF31FC07BF320C07CF321C07DF32E0EE3
:102760007E6F22C07FF323C080F324C081F30C0E60
:10277000BB6F00011A5205E1000E016E03010FD17B
:1027800000011A50E508D8B407D122C0BCF323C019
:10279000BDF324C0BEF30301BC516D0809E0BC5178
:1027A0004D0806E0BC51570803E0BC5177080FE123
:1027B000BD51500809E0BD51700806E0BD51410807
:1027C00003E0BD51610803E1BE51330807E0BE518B
:1027D000560804E0BE517608D8A4DDD0D56B2E5043
:1027E000D525BF6F000E2F20C06FC16BC26BC0C359
:1027F000C2F3BFC3C1F3BF6BC06BD46BD36BD76BDA
:102800003450D7250001FE6F000E03013520000172
:10281000FF6F000E0301D3210101006F000E0301C1
:10282000D4210101016F0301BF510001FE27030103
:10283000C0510001FF230301C15101010023030125
:10284000C251010101230301D56BD46BD36B34C09A
:10285000D2F3D96BD86BD76B35C0D6F3D8C303F09E
:10286000D7C302F035C001F0006A00503424DB6F9A
:102870003550D321DC6FD751D421DD6FD851D5210C
:10288000DE6FE26FDDC3E1F3DCC3E0F3DBC3DFF354
:10289000E66BE56BE46BE1C0E3F3000196EC0BF053
:1028A000E25103010024E06F0001E3510301012024
:1028B000E16F000E0220E26F000E0320E36F0001C3
:1028C000E4510301E0250001EA6FE5510301E12134
:1028D0000001EB6F000E0301E2210001EC6F000E1E
:1028E0000301E3210001ED6F0301D36BEE0EE96EEE
:1028F000D3C3EAFF36C0EFFFD36BEE0ED26F010EEB
:10290000D225016E000ED32101C0E9FFEA6E37C067
:10291000EFFFD36BEE0ED26F020ED225016E000ECA
:10292000D32101C0E9FFEA6E38C0EFFFD36BEE0E92
:10293000D26F030ED225016E000ED32101C0E9FF34
:10294000EA6E39C0EFFF755323E00D0E9EA8FED747
:10295000AD6E0A0E9EA8FED7AD6EBA6BBB51BA5DC6
:102960000FE2036ABA51760FE96E030E0320EA6E96
:10297000EFCFD2F3D2519EA8FED7AD6EBA2BEED7D1
:102980000D0E9EA8FED7AD6E0A0E9EA8FED7AD6EA8
:10299000010E016E04D00001000E016E0301000162
:1029A000000C020E03018D6F8E6B080E8F6F040EEC
:1029B000906F000106EC07F0010E0301E16F0001CA
:1029C0002EEC06F0FF0ED880DC5503018B6FFF0E56
:1029D000D8800001DB5503018C6F020E8D6F0B0E4A
:1029E0008E6F8BC38FF38CC390F3000106EC07F05E
:1029F000010E0301E16F00012EEC06F0010E030150
:102A0000E16F00012EEC06F036EF15F08A96100EFD
:102A100003018D6F8C6B8C5302E18D5312E0976B29
:102A20000001D2EC06F0000E81A4010E03018B150B
:102A300003E00001F8D703018C51D8B48D078C074F
:102A4000EAD78A860001000C03018A6B896B886BC8
:102A5000876B866B856B020E8D6F0B0E8E6FFE0E75
:102A60008F6F906F000106EC07F09BD7FF0ED880A8
:102A7000DC5503018B6FFF0ED8800001DB5503018D
:102A80008C6F020E8D6F0B0E8E6F8BC38FF38CC30A
:102A900090F3000106EC07F003017151755D816F41
:102AA00072517659826F73517759836F7451785987
:102AB000846F74C3A3F373C3A2F372C3A1F371C38E
:102AC000A0F3A76BA66BA56BE1C0A4F30001EEEC2D
:102AD0000FF003C074F302C073F301C072F300C0BF
:102AE00071F378C3A3F377C3A2F376C3A1F375C3DD
:102AF000A0F30301A76BA66BA56BE1C0A4F30001D3
:102B0000EEEC0FF003C078F302C077F301C076F368
:102B100000C075F3F28AE09194948B8403018A6B70
:102B20000001E15103018A5DD8B002EF1AF0010EF5
:102B30008527D8B0862BD8B4872BD8B4882B020E23
:102B40000001FE5D0301796F000E0001FF590301D2
:102B50007A6F000E0101005903017B6F000E010125
:102B6000015903017C6FE1C000F0016A026A036A47
:102B700003C08EF302C08DF301C08CF3E1C08BF370
:102B80007CC3E2F37BC3E1F37AC3E0F379C3DFF301
:102B900003C0E6F302C0E5F301C0E4F3E1C0E3F3F0
:102BA000000196EC0BF003C07CF302C07BF301C084
:102BB0007AF300C079F3FA51030179270001FB5140
:102BC00003017A230001FC5103017B230001FD5125
:102BD00003017C23016A026A036A8A517927015042
:102BE0007A2302507B2303507C238851845DD8A034
:102BF0004BEF19F00FE18751835DD8A04BEF19F02F
:102C000009E18651825DD8A046D304E18151855DFA
:102C1000D8B041D37CC38EF37BC38DF37AC38CF3DE
:102C200079C38BF35FC3C6FFD8908B378C378D3752
:102C30008E37C950FF0EC96EC7A0FED7C950FF0E10
:102C4000C96EC7A0FED78B92C950510EC96EC7A0DE
:102C5000FED7030E946F8B0E936F020E9325016EB9
:102C6000000E9421036E01C0E9FFEA6EEFCF95F3E9
:102C7000C95095C3C9FFC7A0FED7030E946F8B0E32
:102C8000936F010E9325016E000E9421036E01C017
:102C9000E9FFEA6EEFCF95F3C95095C3C9FFC7A00E
:102CA000FED7030E946F8B0E936F94C303F0E96EFF
:102CB00094C3EAFFEFCF95F3C95095C3C9FFC7A0EE
:102CC000FED7C950C96AC7A0FED7C950FF0EC96E4A
:102CD000C7A0FED7E76B020EE96F080EE86FE85356
:102CE00002E1E95312E0C950FF0EC96EC7A0FED73A
:102CF000C9CFEAF3E751EA5D03E1000E016E07D0A8
:102D0000E851D8B4E907E807EAD7010E016E01528D
:102D1000D8A475D0FE0EE76F020EE96F080EE86FBB
:102D2000E85302E1E95312E0C950FF0EC96EC7A093
:102D3000FED7C9CFEAF3E751EA5D03E1000E016E69
:102D400007D0E851D8B4E907E807EAD7010E016EC9
:102D500001523DE18A96906B100E8F6F8F5302E106
:102D600090531AE081B401D0FDD78A9A926B916B8F
:102D700092530CE191511F0809E3C950FF0EC96E2F
:102D8000C7A0FED7912BD8B4922BF2D78A8A8F5145
:102D9000D8B490078F07E2D78A865FC3C6FFC950B1
:102DA000FF0EC96EC7A0FED7C950FF0EC96EC7A0DF
:102DB000FED78B82C950FF0EC96EC7A0FED7C9507F
:102DC000FF0EC96EC7A0FED7000E016E2FD0C950EE
:102DD000FF0EC96EC7A0FED7C950FF0EC96EC7A0AF
:102DE000FED78B82C950FF0EC96EC7A0FED7C9504F
:102DF000FF0EC96EC7A0FED7010E016E17D0C950D5
:102E0000FF0EC96EC7A0FED7C950FF0EC96EC7A07E
:102E1000FED78B82C950FF0EC96EC7A0FED7C9501E
:102E2000FF0EC96EC7A0FED7010E016E012C33D272
:102E3000210E9EA8FED7AD6E7CC38EF37BC38DF3AF
:102E40007AC38CF379C38BF35FC3C6FFD8908B37FB
:102E50008C378D378E37C950FF0EC96EC7A0FED78D
:102E6000C950FF0EC96EC7A0FED78B92C950510E34
:102E7000C96EC7A0FED7030E946F8B0E936F020E20
:102E80009325016E000E9421036E01C0E9FFEA6EE6
:102E9000EFCF95F3C95095C3C9FFC7A0FED7030E66
:102EA000946F8B0E936F010E9325016E000E94218B
:102EB000036E01C0E9FFEA6EEFCF95F3C95095C3E9
:102EC000C9FFC7A0FED7030E946F8B0E936F94C3F8
:102ED00003F0E96E94C3EAFFEFCF95F3C95095C3B1
:102EE000C9FFC7A0FED7C950C96AC7A0FED7C9503D
:102EF000FF0EC96EC7A0FED7E76B020EE96F080E82
:102F0000E86FE85302E1E95312E0C950FF0EC96EC1
:102F1000C7A0FED7C9CFEAF3E751EA5D03E1000E8F
:102F2000016E07D0E851D8B4E907E807EAD7010EE7
:102F3000016E0152D8A475D0FE0EE76F020EE96F44
:102F4000080EE86FE85302E1E95312E0C950FF0EA2
:102F5000C96EC7A0FED7C9CFEAF3E751EA5D03E126
:102F6000000E016E07D0E851D8B4E907E807EAD7A8
:102F7000010E016E01523DE18A96906B100E8F6F2B
:102F80008F5302E190531AE081B401D0FDD78A9AA1
:102F9000926B916B92530CE191511F0809E3C95058
:102FA000FF0EC96EC7A0FED7912BD8B4922BF2D7D3
:102FB0008A8A8F51D8B490078F07E2D78A865FC379
:102FC000C6FFC950FF0EC96EC7A0FED7C950FF0E7D
:102FD000C96EC7A0FED78B82C950FF0EC96EC7A0AD
:102FE000FED7C950FF0EC96EC7A0FED7000E016EF6
:102FF0002FD0C950FF0EC96EC7A0FED7C950FF0E13
:10300000C96EC7A0FED78B82C950FF0EC96EC7A07C
:10301000FED7C950FF0EC96EC7A0FED7010E016EC4
:1030200017D0C950FF0EC96EC7A0FED7C950FF0EFA
:10303000C96EC7A0FED78B82C950FF0EC96EC7A04C
:10304000FED7C950FF0EC96EC7A0FED7010E016E94
:10305000012C21D1400E9EA8FED7AD6E7CC38EF30D
:103060007BC38DF37AC38CF379C38BF35FC3C6FF45
:10307000D8908B378C378D378E37C950FF0EC96E7D
:10308000C7A0FED7C950FF0EC96EC7A0FED78B924E
:10309000C950510EC96EC7A0FED7030E946F8B0E98
:1030A000936F020E9325016E000E9421036E01C0F2
:1030B000E9FFEA6EEFCF95F3C95095C3C9FFC7A0EA
:1030C000FED7030E946F8B0E936F010E9325016E46
:1030D000000E9421036E01C0E9FFEA6EEFCF95F375
:1030E000C95095C3C9FFC7A0FED7030E946F8B0EBE
:1030F000936F94C303F0E96E94C3EAFFEFCF95F3A7
:10310000C95095C3C9FFC7A0FED7C950C96AC7A097
:10311000FED7C950FF0EC96EC7A0FED7E76B020EDF
:10312000E96F080EE86FE85302E1E95312E0C95075
:10313000FF0EC96EC7A0FED7C9CFEAF3E751EA5D1B
:1031400003E1000E016E07D0E851D8B4E907E807A3
:10315000EAD7010E016E0152D8A475D0FE0EE76FBA
:10316000020EE96F080EE86FE85302E1E95312E03E
:10317000C950FF0EC96EC7A0FED7C9CFEAF3E75109
:10318000EA5D03E1000E016E07D0E851D8B4E9070B
:10319000E807EAD7010E016E01523DE18A96906B75
:1031A000100E8F6F8F5302E190531AE081B401D05B
:1031B000FDD78A9A926B916B92530CE191511F0843
:1031C00009E3C950FF0EC96EC7A0FED7912BD8B432
:1031D000922BF2D78A8A8F51D8B490078F07E2D703
:1031E0008A865FC3C6FFC950FF0EC96EC7A0FED74F
:1031F000C950FF0EC96EC7A0FED78B82C950FF0E03
:10320000C96EC7A0FED7C950FF0EC96EC7A0FED7B2
:10321000000E016E2FD0C950FF0EC96EC7A0FED799
:10322000C950FF0EC96EC7A0FED78B82C950FF0ED2
:10323000C96EC7A0FED7C950FF0EC96EC7A0FED782
:10324000010E016E17D0C950FF0EC96EC7A0FED780
:10325000C950FF0EC96EC7A0FED78B82C950FF0EA2
:10326000C96EC7A0FED7C950FF0EC96EC7A0FED752
:10327000010E016E012C0FD08B6B8B5100017AEC8B
:1032800002F003018B2B006E00509EA8FED7AD6E9E
:103290000E0E8B5DF2E10001DA51070850E183B0B8
:1032A00015D0F29A8B9403018B6B000106EC15F09C
:1032B000020E03018D6F0B0E8E6FFE0E8F6F906FDF
:1032C000000106EC07F06E0E016E4ED183B21DD0E8
:1032D000F25306E1F35304E1F45302E1F55315E030
:1032E000F29A8B94020E03018D6F0B0E8E6FFE0E01
:1032F0008F6F906F000106EC07F003018B6B0001EC
:1033000006EC15F0700E016E2FD183BA18D0D00ED6
:10331000DB6FDC6FF29A8B94020E03018D6F0B0E44
:103320008E6FFE0E8F6F906F000106EC07F00301A9
:103330008B6B000106EC15F07A0E016E15D1DA5395
:1033400013E1833C01D00FD0E0A50CD0E095F56BE4
:10335000F46BF36B83CFF2F0E091E0838B946B0E10
:10336000016E02D101D0E085E0AD07D00A0E030165
:10337000E16F00012EEC06F0F7D7DF2D10D0F29AA6
:103380008B94020E03018D6F0B0E8E6FFE0E8F6FEE
:10339000906F000106EC07F0650E016EE5D0E0A12C
:1033A0002DD0F29AE09103018B6B8B5100018FECD1
:1033B00002F003018B2B006E00509EA8FED7AD6E6D
:1033C000160E8B5DF2E10D0E9EA8FED7AD6E0A0EB5
:1033D0009EA8FED7AD6E8B94020E8D6F0B0E8E6F76
:1033E000FE0E8F6F906F000106EC07F003018B6BF0
:1033F000000106EC15F06B0E016EB6D003018A2BAE
:1034000090EF15F00A0E7525006E000E7621016E04
:10341000000E7721026E000E7821036E7451035C5A
:1034200028E30BE17351025C24E307E17251015C74
:1034300020E303E10050715D1CE201C105F100C110
:1034400004F1FFC003F1FEC002F105C1D5F304C1D0
:10345000D4F303C1D3F302C1D2F3000183EC0EF025
:1034600003C001F102C000F101C0FFF000C0FEF096
:103470000301FF0ED8800001DC5503018B6FFF0EA6
:10348000D8800001DB5503018C6F020E8D6F0B0E8F
:103490008E6F8BC38FF38CC390F3000106EC07F0A3
:1034A000DA51070839E183B837D0140E0301E16F10
:1034B00000012EEC06F083B807D0140E0301E16F73
:1034C00000012EEC06F0F7D783A81DD0140E0301DF
:1034D000E16F00012EEC06F0DF2D14D08B94020E6C
:1034E00003018D6F0B0E8E6FFE0E8F6F906F0001BC
:1034F00006EC07F003018B6B000106EC15F0650E7E
:10350000016E32D0E1D783B801D0FDD7140E03018C
:10351000E16F00012EEC06F0FEC07DF3FFC07EF3EC
:1035200000C17FF3010101510F0B0301806F805136
:103530000F0814E3D8A48FEF15F07F51FF080EE3B6
:10354000D8A48FEF15F07E51FF0808E3D8A48FEFC1
:1035500015F07D51EE08D8B08FEF15F0F29A00010A
:10356000E0938B94730E016E000C0301756B0201E6
:103570002CAF04D0010E0301756F02012CAB04D0F7
:10358000010E0301751B02012CA904D0010E0301D9
:10359000751B02012CA504D0010E0301751B02014D
:1035A000D8902C370301755102012C132CC201F065
:1035B0000001000CFF0E0301706F6F6F01011153CA
:1035C00057E1105355E10F510301705DD8B002D09F
:1035D00001014ED005E16F5101010E5D49E2030189
:1035E000010E5B27D8B05C2BD8B45D2BD8B45E2B12
:1035F0000001BBDF010E015C0301716F2C0E712510
:10360000E96E010EEA6ED8B0EA2AEF3C01D01DD077
:103610002C0E7125E96E010EEA6ED8B0EA2AEF5041
:10362000EF2A726F7251F2CF73F3F29E000161ECD8
:1036300000F0030173BFF28E706B6F6F71C36EF396
:103640006D6B6D516F276E5170235E530AE15D53B0
:1036500008E15C51FC080AE2FF0A03E15B51E8085B
:1036600005E2006A016A026A036A09D0A7D701016C
:103670006FC300F070C301F0026A036A0301000126
:1036800070EF31F00301746B0A0EC16EBE0EC06E96
:10369000736B73510F0818E311C103F010C102F0EE
:1036A0000FC101F00EC100F07351756F07E0D890A3
:1036B0000332023201320032752FF9D700A002D056
:1036C00073C374F3732BE5D700014FDF0301716BF4
:1036D00001C070F370C371F3706B000146DF0150DD
:1036E00003017027000E712300000F0E736F7351DA
:1036F000745D16E2036A010E026E7351006E05E0FE
:10370000D89002360336002EFBD70250FF0A006E17
:10371000FF0E031A00507017035071177307E7D795
:103720006F6B6E6B736B7351745D2EE3C282C2A2BA
:1037300001D0FDD7C3A002D0728101D07291090ED1
:10374000006E002EFED700D0C282C2A201D0FDD7EB
:10375000000EC3B0010E756F000E72B1010E755DE3
:1037600012E072A10FD0036A010E026E7351006E57
:1037700005E0D89002360336002EFBD702506E13B8
:1037800003506F13732BCFD770516E1B71516F1B8A
:103790000101115311E110530FE10F5103016F5D4E
:1037A000D8B002D0010108D009E16E5101010E5DCF
:1037B000D8B002D0030102D0000E01D0010E0301E7
:1037C0006D1582E12E0E9EA8FED7AD6E6EC301F080
:1037D0006FC302F0000182EF31F0F86AD09E0D8EC7
:1037E000FE0E006E040E016E020EE96E000EEA6E11
:1037F000EE6A002EFDD7012EFBD7EA6AE96AB88689
:10380000110EAF6E040EB06EA60EAC6E900EAB6EC7
:10381000C150C00B0F09C16E070EB46E8B6A7F0ECC
:10382000926EC50E936E940E946EFF0E956E070EFB
:10383000966E9B8C110EC26E94948B940F0EC16E7B
:1038400080CFDAF0070EDA1780A604D0220E03012B
:103850005F6F03D0200E03015F6F0A0EC16E880EEA
:10386000C06EF19CF19EF292820ED56E8B808A9290
:10387000320EE16F00012EEC06F00D0E9EA8FED771
:10388000AD6E0A0E9EA8FED7AD6E0D0E9EA8FED799
:10389000AD6E0A0E9EA8FED7AD6E03016D6B0001E2
:1038A00043EF06F00D0E9EA8FED7AD6E0A0E9EA841
:1038B000FED7AD6E0D0E9EA8FED7AD6E0A0E9EA869
:1038C000FED7AD6E03016D6B6D510001EEEC00F0A3
:1038D00003016D2B006E00509EA8FED7AD6E2B0E1F
:1038E0006D5DF2E1030E6E6F770E9EA8FED7AD6E92
:1038F0006E2FFAD72B0E6F6F6F510001EEEC00F0B8
:1039000003016F2B006E00509EA8FED7AD6E370EE0
:103910006F5DF2E10D0E9EA8FED7AD6E0A0E9EA859
:10392000FED7AD6E0D0E9EA8FED7AD6E0A0E9EA8F8
:10393000FED7AD6E8B828A888A86C69A320EE16F78
:1039400000012EEC06F08A92FA0E03016D6F000161
:10395000BFEF06F08A82320E0301E16F00012EEC08
:1039600006F0320E0301E16F00012EEC06F081A497
:10397000EAD7A60E006E002EFED70000020E03014D
:103980008D6F8E6B8F6B040E906F000106EC07F04D
:103990000A0E0301E16F00012EEC06F081A4E9D7C5
:1039A000320E0301E16F00012EEC06F0320E03012E
:1039B000E16F00012EEC06F081A4F2D7010E0301A5
:1039C000E16F00012EEC06F0020E03018D6F8E6B8D
:1039D000080E8F6F906B000106EC07F0FF0ED88089
:1039E000DC5503016D6FFF0ED8800001DB5503012C
:1039F0006E6F020E8D6F0B0E8E6F6DC38FF36EC3E5
:103A000090F3000106EC07F0010E0301E16F0001E5
:103A10002EEC06F003016D6B6D51000183EC03F099
:103A2000000907E003016D2B9EA8FED7AD6EF4D709
:103A300000010D0E9EA8FED7AD6E0A0E9EA8FED701
:103A4000AD6E8A888A86E09DDF6BDE6BD00EDC6F00
:103A5000DB6F300EDD6F010E0301616F626B612D54
:103A600001D002D0000E01D0010E6D6F6251090825
:103A700002E2000E01D0010E6D150AE0010EDD6FAD
:103A800000019EEC07F001C061F30301622BE7D750
:103A9000612D11D06D6B6D51000117EC01F0030128
:103AA0006D2B006E00509EA8FED7AD6E290E6D5D89
:103AB000F2E10300FED70001E7EC0BF0E85303E16D
:103AC000E95102081BE003016D6B6D51000139ECF7
:103AD00001F003016D2B006E00509EA8FED7AD6E65
:103AE000130E6D5DF2E10D0E9EA8FED7AD6E0A0EAF
:103AF0009EA8FED7AD6E0001E7EC0BF003016D6BE5
:103B00006D51000150EC01F003016D2B006E00506F
:103B10009EA8FED7AD6E110E6D5DF2E10D0E9EA852
:103B2000FED7AD6E0A0E9EA8FED7AD6E0001F56BF6
:103B3000F46BF36B010EF26F4CEF0FF003016D6B42
:103B40006D51000166EC01F003016D2B006E005019
:103B50009EA8FED7AD6E110E6D5DF2E10EC1E2F3CF
:103B60001B0EE36F00015FEC07F00D0E9EA8FED761
:103B7000AD6E0A0E9EA8FED7AD6E19C109F118C12F
:103B800008F117C107F116C106F1730E0301606F4A
:103B90000001E099E0830301616B0001E091E0978F
:103BA000C00EF212F29A010111530AE1105308E11A
:103BB0000F5100080AE2FF0A03E10E512C0805E24A
:103BC000960E03015A6F09D00101D89011311031BE
:103BD0000F310E31E8CF5AF30301626B5A51625D27
:103BE00011E2D8906235026E036A033602502D0F3F
:103BF000E96E020E0320EA6EFF0EEC6EED52EF6EE0
:103C0000622BECD70D0E9EA8FED7AD6E0A0E9EA8B5
:103C1000FED7AD6E0D0E9EA8FED7AD6E0A0E9EA805
:103C2000FED7AD6E5F51200810E16D6B6D51000144
:103C30007DEC01F003016D2B006E00509EA8FED7B5
:103C4000AD6E390E6D5DF2E10FD06D6B6D510001FF
:103C5000A7EC01F003016D2B006E00509EA8FED76B
:103C6000AD6E120E6D5DF2E10D0E9EA8FED7AD6E2B
:103C70000A0E9EA8FED7AD6E0001DA51030808E0D7
:103C8000DA51020805E0DA510608D8A47BEF25F0E6
:103C90000D0E9EA8FED7AD6E0A0E9EA8FED7AD6E85
:103CA000DA5103081BE103016D6B6D510001BEEC9D
:103CB00001F003016D2B006E00509EA8FED7AD6E83
:103CC000140E6D5DF2E10D0E9EA8FED7AD6E0A0ECC
:103CD0009EA8FED7AD6E9D8A3BD00001DA51060842
:103CE0001BE103016D6B6D510001D6EC01F0030186
:103CF0006D2B006E00509EA8FED7AD6E190E6D5D47
:103D0000F2E10D0E9EA8FED7AD6E0A0E9EA8FED75C
:103D1000AD6E9D8A1DD00001DA5102081AE103013F
:103D20006D6B6D510001F0EC01F003016D2B006E25
:103D300000509EA8FED7AD6E130E6D5DF2E10D0E24
:103D40009EA8FED7AD6E0A0E9EA8FED7AD6EF28875
:103D500000010D0E9EA8FED7AD6E0A0E9EA8FED7DE
:103D6000AD6E010EDE6FE093F56BF46BFF0EF36F3B
:103D7000F26FF3C06EF3F2C06DF36EC370F36DC3F8
:103D80006FF303019B6B70C3D3F36FC3D2F3270EA2
:103D9000D56F100ED46F0001CBEC0FF001C07CF397
:103DA00003019F6B9E6B9D6B7CC39CF39FC3E2F3EF
:103DB0009EC3E1F39DC3E0F37CC3DFF3E66BE56BE9
:103DC000270EE46F100EE36F000196EC0BF003C0BA
:103DD0008AF302C089F301C088F300C087F30301AE
:103DE00087516F5D9C6F885170599D6F000E89558A
:103DF0009E6F000E8A559F6FA36F9EC3A2F39DC353
:103E0000A1F39CC3A0F3A76BA66B030EA56FE80EEE
:103E1000A46F0001EEEC0FF000C07BF303019F6B79
:103E20009E6B9D6B7BC39CF39FC3E2F39EC3E1F348
:103E30009DC3E0F37BC3DFF3E66BE56B030EE46F3A
:103E4000E80EE36F000196EC0BF0005003018727AA
:103E5000015088230250892303508A2387516F5DC4
:103E60009C6F885170599D6F000E89559E6F000E92
:103E70008A559F6FA36F9EC3A2F39DC3A1F39CC3FA
:103E8000A0F3A76BA66BA56B640EA46F0001EEEC0C
:103E90000FF000C077F303019F6B9E6B9D6B77C3A0
:103EA0009CF39FC3E2F39EC3E1F39DC3E0F377C3AA
:103EB000DFF3E66BE56BE46B640EE36F000196ECF9
:103EC0000BF00050030187270150882302508923FB
:103ED00003508A2387516F5D9C6F885170599D6F85
:103EE000000E89559E6F000E8A559F6FA36F9EC36B
:103EF000A2F39DC3A1F39CC3A0F3A76BA66BA56B14
:103F00000A0EA46F0001EEEC0FF000C076F303017F
:103F10009F6B9E6B9D6B76C39CF39FC3E2F39EC326
:103F2000E1F39DC3E0F376C3DFF3E66BE56BE46B8F
:103F30000A0EE36F000196EC0BF000500301872797
:103F4000015088230250892303508A2387516F5DD3
:103F5000756F9A6B996B986B976B19C109F118C1C2
:103F600008F117C107F116C106F19A31926F993124
:103F7000916F9831906F97318F6F92339133903367
:103F80008F339233913390338F3392339133903315
:103F90008F330F0E921792C396F391C395F390C38C
:103FA00094F38FC393F392C3A3F391C3A2F390C38B
:103FB000A1F38FC3A0F3A76BA66BA56BE1C0A4F31D
:103FC0000001EEEC0FF003C092F302C091F301C0C8
:103FD00090F300C08FF392C3E2F391C3E1F390C377
:103FE000E0F38FC3DFF30301E66BE56BE46BE1C045
:103FF000E3F3000196EC0BF003C08EF302C08DF3E7
:1040000001C08CF300C08BF303018B51935D8B6F68
:104010008C5194598C6F8D5195598D6F8E51965945
:104020008E6F8F5306E1905304E1915302E1925356
:1040300025E009C10DF108C10CF107C10BF106C162
:104040000AF10DC1D5F30CC1D4F30BC1D3F30AC1EE
:10405000D2F3000183EC0EF003C009F102C008F1B5
:1040600001C007F100C006F1FF0E03018F27D8A0A1
:104070009027D8A09127D8A09227D3D7020E01016C
:10408000065D03017F6F000E010107590301806F78
:10409000000E010108590301816F000E0101095949
:1040A0000301826FE1C000F0016A026A036A03C083
:1040B0009FF302C09EF301C09DF3E1C09CF382C355
:1040C000E2F381C3E1F380C3E0F37FC3DFF303C016
:1040D000E6F302C0E5F301C0E4F3E1C0E3F300015D
:1040E00096EC0BF003C082F302C081F301C080F3B1
:1040F00000C07FF3FA5103017F270001FB51030148
:1041000080230001FC51030181230001FD510301C3
:1041100082238B517F278C5180238D5181238E5197
:10412000822382C3E0F381C3DFF380C3DEF37FC366
:10413000DDF3000198EC0AF0100E0301746F745364
:10414000D8B49CD0000171EC0BF003019B2B1852EA
:1041500003E01850E50809E10F0EDE6F000160EC86
:104160000BF00F0E03019B277FD0300E185C7E6F83
:10417000300E195C7D6F000171EC0BF003019B2B7D
:10418000300E185C7A6F300E195C796F000171EC9B
:104190000BF003019B2B300E185C786F7D517B5D1B
:1041A00057E17E517C5D54E17851755D51E1795163
:1041B000765D4EE17A51775D4BE1000171EC0BF0D9
:1041C00071EC0BF018C071F319C072F371EC0BF0C5
:1041D000030E03019B2718C073F371516D0809E0AA
:1041E00071514D0806E07151570803E0715177088D
:1041F0000FE17251500809E07251700806E07251E7
:10420000410803E07251610803E17351330806E08D
:104210007351560803E07351760819E1000ED880F7
:104220009B559C6F010ED8A0E8069D6F9CC3DEF3E2
:10423000000160EC0BF080EC0BF097C300F098C32A
:1042400001F099C302F09AC303F065D0030106D0D0
:10425000030EDE6F000160EC0BF003010A0EDE6F4F
:10426000000160EC0BF00301010E9727D8B0982BEA
:10427000D8B4992BD8B49A2B740761D706C183F3AD
:1042800007C184F308C185F3010109510F0B030134
:10429000866F000180EC0BF003019A510101115D62
:1042A00030E311E1030199510101105D2AE30BE1B3
:1042B0000301985101010F5D24E305E103019751CA
:1042C00001010E5D1EE3030186510F08D8B002D034
:1042D000010117D0D8A441D68551FF08D8B002D02B
:1042E00001010FD0D8A439D68451FF08D8B002D02C
:1042F000010107D0D8A431D68351EF08D8B02DD60C
:10430000010100002D0E9EA8FED7AD6E006A016A65
:10431000026A036A000103C068F302C067F301C0C8
:1043200066F300C065F3E0B90DD0E0B30BD0640EC6
:104330000301E16F00012EEC06F02E0E9EA8FED7C1
:10434000AD6EF1D7F3C06EF3F2C06DF36EC370F3D0
:104350006DC36FF303019B6B70C3D3F36FC3D2F3D1
:10436000270ED56F100ED46F0001CBEC0FF001C0FB
:104370007CF303019F6B9E6B9D6B7CC39CF39FC37F
:10438000E2F39EC3E1F39DC3E0F37CC3DFF3E66B8E
:10439000E56B270EE46F100EE36F000196EC0BF057
:1043A00003C08AF302C089F301C088F300C087F319
:1043B000030187516F5D9C6F885170599D6F000E8E
:1043C00089559E6F000E8A559F6FA36F9EC3A2F3FF
:1043D0009DC3A1F39CC3A0F3A76BA66B030EA56FAF
:1043E000E80EA46F0001EEEC0FF000C07BF30301B8
:1043F0009F6B9E6B9D6B7BC39CF39FC3E2F39EC33D
:10440000E1F39DC3E0F37BC3DFF3E66BE56B030EE3
:10441000E46FE80EE36F000196EC0BF0005003012F
:104420008727015088230250892303508A2387510C
:104430006F5D9C6F885170599D6F000E89559E6FFE
:10444000000E8A559F6FA36F9EC3A2F39DC3A1F375
:104450009CC3A0F3A76BA66BA56B640EA46F0001B1
:10446000EEEC0FF000C077F303019F6B9E6B9D6B2A
:1044700077C39CF39FC3E2F39EC3E1F39DC3E0F3D4
:1044800077C3DFF3E66BE56BE46B640EE36F00016B
:1044900096EC0BF00050030187270150882302504F
:1044A000892303508A2387516F5D9C6F885170590F
:1044B0009D6F000E89559E6F000E8A559F6FA36FEA
:1044C0009EC3A2F39DC3A1F39CC3A0F3A76BA66BED
:1044D000A56B0A0EA46F0001EEEC0FF000C076F39E
:1044E00003019F6B9E6B9D6B76C39CF39FC3E2F3AE
:1044F0009EC3E1F39DC3E0F376C3DFF3E66BE56BA8
:10450000E46B0A0EE36F000196EC0BF00050030120
:104510008727015088230250892303508A2387511B
:104520006F5D756F9A6B996B986B976B19C109F1F9
:1045300018C108F117C107F116C106F19A31926F3F
:104540009931916F9831906F97318F6F923391338A
:1045500090338F339233913390338F33923391333F
:1045600090338F330F0E921792C396F391C395F346
:1045700090C394F38FC393F392C3A3F391C3A2F3B5
:1045800090C3A1F38FC3A0F3A76BA66BA56BE1C08B
:10459000A4F30001EEEC0FF003C092F302C091F31C
:1045A00001C090F300C08FF392C3E2F391C3E1F333
:1045B00090C3E0F38FC3DFF30301E66BE56BE46BBD
:1045C000E1C0E3F3000196EC0BF003C08EF302C0F0
:1045D0008DF301C08CF300C08BF303018B51935D0D
:1045E0008B6F8C5194598C6F8D5195598D6F8E5165
:1045F00096598E6F8F5306E1905304E1915302E177
:10460000925325E009C10DF108C10CF107C10BF16E
:1046100006C10AF10DC1D5F30CC1D4F30BC1D3F31C
:104620000AC1D2F3000183EC0EF003C009F102C00D
:1046300008F101C007F100C006F1FF0E03018F274A
:10464000D8A09027D8A09127D8A09227D3D7020E20
:104650000101065D03017F6F000E0101075903018F
:10466000806F000E010108590301816F000E0101E6
:1046700009590301826FE1C000F0016A026A036A0E
:1046800003C09FF302C09EF301C09DF3E1C09CF301
:1046900082C3E2F381C3E1F380C3E0F37FC3DFF3BE
:1046A00003C0E6F302C0E5F301C0E4F3E1C0E3F3C5
:1046B000000196EC0BF003C082F302C081F301C04D
:1046C00080F300C07FF3FA5103017F270001FB5103
:1046D000030180230001FC51030181230001FD51EE
:1046E000030182238B517F278C5180238D5181239D
:1046F0008E51822382C3E0F381C3DFF380C3DEF3F4
:104700007FC3DDF3000198EC0AF0100E0301746F13
:104710007453D8B49CD0000171EC0BF003019B2BB7
:10472000185203E01850E50809E10F0EDE6F000192
:1047300060EC0BF00F0E03019B277FD0300E185C4E
:104740007E6F300E195C7D6F000171EC0BF0030180
:104750009B2B300E185C7A6F300E195C796F00015C
:1047600071EC0BF003019B2B300E185C786F7D51C0
:104770007B5D57E17E517C5D54E17851755D51E17F
:104780007951765D4EE17A51775D4BE1000171EC34
:104790000BF071EC0BF018C071F319C072F371ECEF
:1047A0000BF0030E03019B2718C073F371516D08C2
:1047B00009E071514D0806E07151570803E071514D
:1047C00077080FE17251500809E07251700806E055
:1047D0007251410803E07251610803E173513308DB
:1047E00006E07351560803E07351760819E1000E94
:1047F000D8809B559C6F010ED8A0E8069D6F9CC386
:10480000DEF3000160EC0BF080EC0BF097C300F0DE
:1048100098C301F099C302F09AC303F065D0030175
:1048200006D0030EDE6F000160EC0BF003010A0EF0
:10483000DE6F000160EC0BF00301010E9727D8B08A
:10484000982BD8B4992BD8B49A2B740761D706C18A
:1048500083F307C184F308C185F3010109510F0BEC
:104860000301866F000180EC0BF003019A510101F6
:10487000115D30E311E1030199510101105D2AE35B
:104880000BE10301985101010F5D24E305E10301F0
:10489000975101010E5D1EE3030186510F08D8B048
:1048A00002D0010117D0D8A441D68551FF08D8B055
:1048B00002D001010FD0D8A439D68451FF08D8B056
:1048C00002D0010107D0D8A431D68351EF08D8B067
:1048D0002DD6010100002D0E9EA8FED7AD6E006AF8
:1048E000016A026A036A000103C068F302C067F349
:1048F00001C066F300C065F30301655307E1665329
:1049000005E1675303E16853D8B4F3D0685307E176
:10491000675305E1665303E16551040818E2050E8B
:10492000655D6D6F000E66596E6F000E67596F6F93
:10493000000E6859706F746F6FC373F36EC372F3B8
:104940006DC371F3756B000140EC10F00301685307
:1049500007E1675305E1665303E16551030818E277
:10496000040E655D6D6F000E66596E6F000E67591F
:104970006F6F000E6859706F746F6FC373F36EC3FF
:1049800072F36DC371F3756B000140EC10F003011D
:10499000685307E1675305E1665303E16551020877
:1049A00018E2030E655D6D6F000E66596E6F000EA6
:1049B00067596F6F000E6859706F746F6FC373F330
:1049C0006EC372F36DC371F3756B000140EC10F0B0
:1049D0000301685307E1675305E1665303E165513D
:1049E000010818E2020E655D6D6F000E66596E6F6C
:1049F000000E67596F6F000E6859706F746F6FC348
:104A000073F36EC372F36DC371F3756B000140EC09
:104A100010F00301655306E1665304E1675302E1B8
:104A2000685318E0010E655D6D6F000E66596E6F7C
:104A3000000E67596F6F000E6859706F746F6FC307
:104A400073F36EC372F36DC371F3756B000140ECC9
:104A500010F0030168C374F367C373F366C372F3A2
:104A600065C371F3010E756F000140EC10F00D0E7F
:104A70009EA8FED7AD6E0A0E9EA8FED7AD6ED8904A
:104A8000036AF131026EF031016EEF31006EEA25FA
:104A900003016D6F01500001EB2103016E6F0250A5
:104AA0000001EC2103016F6F03500001ED210301B0
:104AB000706FEDC074F3ECC073F3EBC072F3EAC037
:104AC00071F3786F6FC377F36EC376F36DC375F3CD
:104AD000000124EC15F001C060F3E0A904D0E0B3BC
:104AE00002D0030113D7010E0301E16F00012EEC88
:104AF00006F0000118D4DA53D8A452EF29F00301CC
:104B00006D6B6D51000107EC02F003016D2B006E1F
:104B100000509EA8FED7AD6E130E6D5DF2E10D0E36
:104B20009EA8FED7AD6E0A0E9EA8FED7AD6E000100
:104B3000E093010EDE6FE0B305D0F56BF46BF36B21
:104B400083CFF2F00301686B676B666B656B0001E6
:104B5000F251FE080CE1F3530AE1F45308E1F55376
:104B600006E103016C6B6B6B6A6B696B0001F251C0
:104B7000FD080DE1F3530BE1F45309E1F55307E1AF
:104B800003016C6B6B6B6A6B010E696F0001F25174
:104B9000FB080DE1F3530BE1F45309E1F55307E191
:104BA00003016C6B6B6B6A6B020E696F0001F25153
:104BB000F7080DE1F3530BE1F45309E1F55307E175
:104BC00003016C6B6B6B6A6B030E696F0001F25132
:104BD000EF080DE1F3530BE1F45309E1F55307E15D
:104BE00003016C6B6B6B6A6B040E696F0001F25111
:104BF000DF080DE1F3530BE1F45309E1F55307E14D
:104C000003016C6B6B6B6A6B050E696F0001F251EF
:104C1000BF080DE1F3530BE1F45309E1F55307E14C
:104C200003016C6B6B6B6A6B060E696F0001F251CE
:104C30007F080DE1F3530BE1F45309E1F55307E16C
:104C400003016C6B6B6B6A6B070E696F0001F23DC1
:104C500007D0F35305E1F45303E1F553D8B4DAD2A6
:104C60006AC36EF369C36DF36EC370F36DC36FF304
:104C700003019B6B70C3D3F36FC3D2F3270ED56FC1
:104C8000100ED46F0001CBEC0FF001C07CF30301D8
:104C90009F6B9E6B9D6B7CC39CF39FC3E2F39EC393
:104CA000E1F39DC3E0F37CC3DFF3E66BE56B270E16
:104CB000E46F100EE36F000196EC0BF003C08AF373
:104CC00002C089F301C088F300C087F30301875154
:104CD0006F5D9C6F885170599D6F000E89559E6F56
:104CE000000E8A559F6FA36F9EC3A2F39DC3A1F3CD
:104CF0009CC3A0F3A76BA66B030EA56FE80EA46F71
:104D00000001EEEC0FF000C07BF303019F6B9E6B84
:104D10009D6B7BC39CF39FC3E2F39EC3E1F39DC3F2
:104D2000E0F37BC3DFF3E66BE56B030EE46FE80EA5
:104D3000E36F000196EC0BF0005003018727015050
:104D400088230250892303508A2387516F5D9C6F0B
:104D5000885170599D6F000E89559E6F000E8A55BF
:104D60009F6FA36F9EC3A2F39DC3A1F39CC3A0F347
:104D7000A76BA66BA56B640EA46F0001EEEC0FF0A1
:104D800000C077F303019F6B9E6B9D6B77C39CF311
:104D90009FC3E2F39EC3E1F39DC3E0F377C3DFF368
:104DA000E66BE56BE46B640EE36F000196EC0BF0D1
:104DB00000500301872701508823025089230350A4
:104DC0008A2387516F5D9C6F885170599D6F000ECB
:104DD00089559E6F000E8A559F6FA36F9EC3A2F3E5
:104DE0009DC3A1F39CC3A0F3A76BA66BA56B0A0E92
:104DF000A46F0001EEEC0FF000C076F303019F6B8F
:104E00009E6B9D6B76C39CF39FC3E2F39EC3E1F35D
:104E10009DC3E0F376C3DFF3E66BE56BE46B0A0E4C
:104E2000E36F000196EC0BF000500301872701505F
:104E300088230250892303508A2387516F5D756F41
:104E40009A6B996B986B976B19C109F118C108F1AE
:104E500017C107F116C106F19A31926F9931916F1E
:104E60009831906F97318F6F9233913390338F33A6
:104E70009233913390338F339233913390338F3316
:104E80000F0E921792C396F391C395F390C394F3C8
:104E90008FC393F392C3A3F391C3A2F390C3A1F37F
:104EA0008FC3A0F3A76BA66BA56BE1C0A4F30001B1
:104EB000EEEC0FF003C092F302C091F301C090F347
:104EC00000C08FF392C3E2F391C3E1F390C3E0F328
:104ED0008FC3DFF30301E66BE56BE46BE1C0E3F343
:104EE000000196EC0BF003C08EF302C08DF301C0FD
:104EF0008CF300C08BF303018B51935D8B6F8C514E
:104F000094598C6F8D5195598D6F8E5196598E6F26
:104F10008F5306E1905304E1915302E1925325E04F
:104F200009C10DF108C10CF107C10BF106C10AF16D
:104F30000DC1D5F30CC1D4F30BC1D3F30AC1D2F325
:104F4000000183EC0EF003C009F102C008F101C0BA
:104F500007F100C006F1FF0E03018F27D8A09027AC
:104F6000D8A09127D8A09227D3D7020E0101065DC1
:104F700003017F6F000E010107590301806F000ECE
:104F8000010108590301816F000E01010959030154
:104F9000826FE1C000F0016A026A036A03C09FF3F6
:104FA00002C09EF301C09DF3E1C09CF382C3E2F313
:104FB00081C3E1F380C3E0F37FC3DFF303C0E6F313
:104FC00002C0E5F301C0E4F3E1C0E3F3000196ECB5
:104FD0000BF003C082F302C081F301C080F300C074
:104FE0007FF3FA5103017F270001FB510301802366
:104FF0000001FC51030181230001FD5103018223C3
:105000008B517F278C5180238D5181238E51822398
:1050100082C3E0F381C3DFF380C3DEF37FC3DDF33C
:10502000000198EC0AF0100E0301746F7453D8B4A9
:105030009CD0000171EC0BF003019B2B185203E094
:105040001850E50809E10F0EDE6F000160EC0BF06F
:105050000F0E03019B277FD0300E185C7E6F300E41
:10506000195C7D6F000171EC0BF003019B2B300E7E
:10507000185C7A6F300E195C796F000171EC0BF0DF
:1050800003019B2B300E185C786F7D517B5D57E1DF
:105090007E517C5D54E17851755D51E17951765DC9
:1050A0004EE17A51775D4BE1000171EC0BF071EC50
:1050B0000BF018C071F319C072F371EC0BF0030E12
:1050C00003019B2718C073F371516D0809E07151FA
:1050D0004D0806E07151570803E0715177080FE160
:1050E0007251500809E07251700806E0725141088F
:1050F00003E07251610803E17351330806E0735114
:10510000560803E07351760819E1000ED8809B55CC
:105110009C6F010ED8A0E8069D6F9CC3DEF30001D2
:1051200060EC0BF080EC0BF097C300F098C301F03B
:1051300099C302F09AC303F065D0030106D0030EB1
:10514000DE6F000160EC0BF003010A0EDE6F000160
:1051500060EC0BF00301010E9727D8B0982BD8B460
:10516000992BD8B49A2B740761D706C183F307C172
:1051700084F308C185F3010109510F0B0301866F08
:10518000000180EC0BF003019A510101115D30E345
:1051900011E1030199510101105D2AE30BE10301C3
:1051A000985101010F5D24E305E1030197510101CD
:1051B0000E5D1EE3030186510F08D8B002D0010135
:1051C00017D0D8A441D68551FF08D8B002D001012C
:1051D0000FD0D8A439D68451FF08D8B002D001012D
:1051E00007D0D8A431D68351EF08D8B02DD601010D
:1051F00000002D0E9EA8FED7AD6E006A016A026AFD
:10520000036A000103C068F302C067F301C066F3DC
:1052100000C065F30301655306E1665304E167537B
:1052200002E168533CE068C374F367C373F366C379
:1052300072F365C371F3756B000140EC10F0E093FD
:10524000D890036AF131026EF031016EEF31006ED9
:10525000EA2503016D6F01500001EB2103016E6F20
:1052600002500001EC2103016F6F03500001ED219A
:105270000301706FEDC074F3ECC073F3EBC072F315
:10528000EAC071F3786F6FC377F36EC376F36DC3C3
:1052900075F3000124EC15F001C060F302D00001A9
:1052A000E09347D4DA2D3EEF2DF003016D6B6D5185
:1052B00000011EEC02F003016D2B006E00509EA851
:1052C000FED7AD6E110E6D5DF2E10D0E9EA8FED7FC
:1052D000AD6E0A0E9EA8FED7AD6EF288F28A010E60
:1052E0000001DE6FE0B701D0FDD7F3C06EF3F2C06E
:1052F0006DF36EC370F36DC36FF303019B6B70C3EB
:10530000D3F36FC3D2F3270ED56F100ED46F000105
:10531000CBEC0FF001C07CF303019F6B9E6B9D6B88
:105320007CC39CF39FC3E2F39EC3E1F39DC3E0F310
:105330007CC3DFF3E66BE56B270EE46F100EE36FC3
:10534000000196EC0BF003C08AF302C089F301C0A0
:1053500088F300C087F3030187516F5D9C6F88510C
:1053600070599D6F000E89559E6F000E8A559F6F74
:10537000A36F9EC3A2F39DC3A1F39CC3A0F3A76B2D
:10538000A66B030EA56FE80EA46F0001EEEC0FF004
:1053900000C07BF303019F6B9E6B9D6B7BC39CF3F3
:1053A0009FC3E2F39EC3E1F39DC3E0F37BC3DFF34E
:1053B000E66BE56B030EE46FE80EE36F000196EC1D
:1053C0000BF00050030187270150882302508923E6
:1053D00003508A2387516F5D9C6F885170599D6F70
:1053E000000E89559E6F000E8A559F6FA36F9EC356
:1053F000A2F39DC3A1F39CC3A0F3A76BA66BA56BFF
:10540000640EA46F0001EEEC0FF000C077F303010F
:105410009F6B9E6B9D6B77C39CF39FC3E2F39EC310
:10542000E1F39DC3E0F377C3DFF3E66BE56BE46B79
:10543000640EE36F000196EC0BF000500301872728
:10544000015088230250892303508A2387516F5DBE
:105450009C6F885170599D6F000E89559E6F000E8C
:105460008A559F6FA36F9EC3A2F39DC3A1F39CC3F4
:10547000A0F3A76BA66BA56B0A0EA46F0001EEEC60
:105480000FF000C076F303019F6B9E6B9D6B76C39C
:105490009CF39FC3E2F39EC3E1F39DC3E0F376C3A5
:1054A000DFF3E66BE56BE46B0A0EE36F000196EC4D
:1054B0000BF00050030187270150882302508923F5
:1054C00003508A2387516F5D756F9A6B996B986B48
:1054D000976B19C109F118C108F117C107F116C17D
:1054E00006F19A31926F9931916F9831906F97319F
:1054F0008F6F9233913390338F3392339133903354
:105500008F339233913390338F330F0E921792C3B0
:1055100096F391C395F390C394F38FC393F392C31F
:10552000A3F391C3A2F390C3A1F38FC3A0F3A76B1E
:10553000A66BA56BE1C0A4F30001EEEC0FF003C075
:1055400092F302C091F301C090F300C08FF392C3B5
:10555000E2F391C3E1F390C3E0F38FC3DFF3030100
:10556000E66BE56BE46BE1C0E3F3000196EC0BF056
:1055700003C08EF302C08DF301C08CF300C08BF327
:1055800003018B51935D8B6F8C5194598C6F8D51AE
:1055900095598D6F8E5196598E6F8F5306E19053AA
:1055A00004E1915302E1925325E009C10DF108C1D4
:1055B0000CF107C10BF106C10AF10DC1D5F30CC105
:1055C000D4F30BC1D3F30AC1D2F3000183EC0EF084
:1055D00003C009F102C008F101C007F100C006F1E3
:1055E000FF0E03018F27D8A09027D8A09127D8A01D
:1055F0009227D3D7020E0101065D03017F6F000ED3
:10560000010107590301806F000E010108590301D0
:10561000816F000E010109590301826FE1C000F0A2
:10562000016A026A036A03C09FF302C09EF301C0CD
:105630009DF3E1C09CF382C3E2F381C3E1F380C335
:10564000E0F37FC3DFF303C0E6F302C0E5F301C07C
:10565000E4F3E1C0E3F3000196EC0BF003C082F346
:1056600002C081F301C080F300C07FF3FA5103014F
:105670007F270001FB51030180230001FC5103013E
:1056800081230001FD51030182238B517F278C511F
:1056900080238D5181238E51822382C3E0F381C305
:1056A000DFF380C3DEF37FC3DDF3000198EC0AF083
:1056B000100E0301746F7453D8B49CD0000171ECC8
:1056C0000BF003019B2B185203E01850E50809E189
:1056D0000F0EDE6F000160EC0BF00F0E03019B2735
:1056E0007FD0300E185C7E6F300E195C7D6F00012C
:1056F00071EC0BF003019B2B300E185C7A6F300EAF
:10570000195C796F000171EC0BF003019B2B300EDB
:10571000185C786F7D517B5D57E17E517C5D54E173
:105720007851755D51E17951765D4EE17A51775D41
:105730004BE1000171EC0BF071EC0BF018C071F350
:1057400019C072F371EC0BF0030E03019B2718C014
:1057500073F371516D0809E071514D0806E0715104
:10576000570803E0715177080FE17251500809E0C2
:105770007251700806E07251410803E072516108ED
:1057800003E17351330806E07351560803E0735187
:10579000760819E1000ED8809B559C6F010ED8A0A9
:1057A000E8069D6F9CC3DEF3000160EC0BF080EC1B
:1057B0000BF097C300F098C301F099C302F09AC3AD
:1057C00003F065D0030106D0030EDE6F000160EC2C
:1057D0000BF003010A0EDE6F000160EC0BF0030119
:1057E000010E9727D8B0982BD8B4992BD8B49A2B00
:1057F000740761D706C183F307C184F308C185F339
:10580000010109510F0B0301866F000180EC0BF0C1
:1058100003019A510101115D30E311E10301995136
:105820000101105D2AE30BE10301985101010F5DB5
:1058300024E305E10301975101010E5D1EE303011D
:1058400086510F08D8B002D0010117D0D8A441D694
:105850008551FF08D8B002D001010FD0D8A439D6A5
:105860008451FF08D8B002D0010107D0D8A431D6A6
:105870008351EF08D8B02DD6010100002D0E9EA84F
:10588000FED7AD6E006A016A026A036A000103C0B6
:1058900068F302C067F301C066F300C065F303015B
:1058A000655307E1665305E1675303E16853D8B4D4
:1058B000DFD0685307E1675305E1665303E16551A3
:1058C000040818E2050E655D6D6F000E66596E6F77
:1058D000000E67596F6F000E6859706F746F6FC359
:1058E00073F36EC372F36DC371F3756B000140EC1B
:1058F00010F00301685307E1675305E1665303E1C4
:105900006551030818E2040E655D6D6F000E66595F
:105910006E6F000E67596F6F000E6859706F746F6D
:105920006FC373F36EC372F36DC371F3756B0001D4
:1059300040EC10F00301685307E1675305E166533B
:1059400003E16551020818E2030E655D6D6F000EFC
:1059500066596E6F000E67596F6F000E6859706F51
:10596000746F6FC373F36EC372F36DC371F3756BB2
:10597000000140EC10F00301685307E1675305E1B3
:10598000665303E16551010818E2020E655D6D6F13
:10599000000E66596E6F000E67596F6F000E6859E2
:1059A000706F746F6FC373F36EC372F36DC371F373
:1059B000756B000140EC10F00301655306E166537E
:1059C00004E1675302E1685318E0010E655D6D6FF5
:1059D000000E66596E6F000E67596F6F000E6859A2
:1059E000706F746F6FC373F36EC372F36DC371F333
:1059F000756B000140EC10F0030168C374F367C3DA
:105A000073F366C372F365C371F3010E756F000122
:105A100040EC10F0D890036AF131026EF031016E63
:105A2000EF31006EEA2503016D6F01500001EB219B
:105A300003016E6F02500001EC2103016F6F0350F0
:105A40000001ED210301706FEDC074F3ECC073F33E
:105A5000EBC072F3EAC071F3786F6FC377F36EC374
:105A600076F36DC375F3000124EC15F001C060F30B
:105A70000001E0B701D0FDD7E09737D4DA51040830
:105A8000D8A42CEF31F003016D6B6D51000134ECA3
:105A900002F003016D2B006E00509EA8FED7AD6E84
:105AA000150E6D5DF2E10D0E9EA8FED7AD6E0A0ECD
:105AB0009EA8FED7AD6EF288F28A010E0001DE6F5D
:105AC000E0B701D0FDD7F3C06EF3F2C06DF36EC343
:105AD00070F36DC36FF303019B6B70C3D3F36FC39C
:105AE000D2F3270ED56F100ED46F0001CBEC0FF060
:105AF00001C07CF303019F6B9E6B9D6B7CC39CF389
:105B00009FC3E2F39EC3E1F39DC3E0F37CC3DFF3E5
:105B1000E66BE56B270EE46F100EE36F000196EC69
:105B20000BF003C08AF302C089F301C088F300C000
:105B300087F3030187516F5D9C6F885170599D6F8A
:105B4000000E89559E6F000E8A559F6FA36F9EC3EE
:105B5000A2F39DC3A1F39CC3A0F3A76BA66B030E96
:105B6000A56FE80EA46F0001EEEC0FF000C07BF310
:105B700003019F6B9E6B9D6B7BC39CF39FC3E2F302
:105B80009EC3E1F39DC3E0F37BC3DFF3E66BE56BFC
:105B9000030EE46FE80EE36F000196EC0BF000508B
:105BA00003018727015088230250892303508A2349
:105BB00087516F5D9C6F885170599D6F000E89559C
:105BC0009E6F000E8A559F6FA36F9EC3A2F39DC365
:105BD000A1F39CC3A0F3A76BA66BA56B640EA46F87
:105BE0000001EEEC0FF000C077F303019F6B9E6B9A
:105BF0009D6B77C39CF39FC3E2F39EC3E1F39DC308
:105C0000E0F377C3DFF3E66BE56BE46B640EE36F01
:105C1000000196EC0BF00050030187270150882308
:105C20000250892303508A2387516F5D9C6F8851EE
:105C300070599D6F000E89559E6F000E8A559F6F9B
:105C4000A36F9EC3A2F39DC3A1F39CC3A0F3A76B54
:105C5000A66BA56B0A0EA46F0001EEEC0FF000C05E
:105C600076F303019F6B9E6B9D6B76C39CF39FC382
:105C7000E2F39EC3E1F39DC3E0F376C3DFF3E66B8B
:105C8000E56BE46B0A0EE36F000196EC0BF000503D
:105C900003018727015088230250892303508A2358
:105CA00087516F5D756F9A6B996B986B976B19C184
:105CB00009F118C108F117C107F116C106F19A31AF
:105CC000926F9931916F9831906F97318F6F9233B6
:105CD000913390338F339233913390338F339233A8
:105CE000913390338F330F0E921792C396F391C373
:105CF00095F390C394F38FC393F392C3A3F391C32B
:105D0000A2F390C3A1F38FC3A0F3A76BA66BA56BFF
:105D1000E1C0A4F30001EEEC0FF003C092F302C067
:105D200091F301C090F300C08FF392C3E2F391C3EB
:105D3000E1F390C3E0F38FC3DFF30301E66BE56BA0
:105D4000E46BE1C0E3F3000196EC0BF003C08EF3CB
:105D500002C08DF301C08CF300C08BF303018B51A3
:105D6000935D8B6F8C5194598C6F8D5195598D6FBC
:105D70008E5196598E6F8F5306E1905304E19153E3
:105D800002E1925325E009C10DF108C10CF107C1F0
:105D90000BF106C10AF10DC1D5F30CC1D4F30BC14F
:105DA000D3F30AC1D2F3000183EC0EF003C009F172
:105DB00002C008F101C007F100C006F1FF0E0301A7
:105DC0008F27D8A09027D8A09127D8A09227D3D7E3
:105DD000020E0101065D03017F6F000E01010759EC
:105DE0000301806F000E010108590301816F000E4D
:105DF000010109590301826FE1C000F0016A026AE2
:105E0000036A03C09FF302C09EF301C09DF3E1C08B
:105E10009CF382C3E2F381C3E1F380C3E0F37FC369
:105E2000DFF303C0E6F302C0E5F301C0E4F3E1C031
:105E3000E3F3000196EC0BF003C082F302C081F3A0
:105E400001C080F300C07FF3FA5103017F270001F6
:105E5000FB51030180230001FC5103018123000158
:105E6000FD51030182238B517F278C5180238D515B
:105E700081238E51822382C3E0F381C3DFF380C389
:105E8000DEF37FC3DDF3000198EC0AF0100E03018E
:105E9000746F7453D8B49CD0000171EC0BF0030103
:105EA0009B2B185203E01850E50809E10F0EDE6F36
:105EB000000160EC0BF00F0E03019B277FD0300E2A
:105EC000185C7E6F300E195C7D6F000171EC0BF079
:105ED00003019B2B300E185C7A6F300E195C796FC2
:105EE000000171EC0BF003019B2B300E185C786FF6
:105EF0007D517B5D57E17E517C5D54E17851755D4C
:105F000051E17951765D4EE17A51775D4BE10001C7
:105F100071EC0BF071EC0BF018C071F319C072F357
:105F200071EC0BF0030E03019B2718C073F3715142
:105F30006D0809E071514D0806E07151570803E002
:105F4000715177080FE17251500809E072517008E1
:105F500006E07251410803E07251610803E1735198
:105F6000330806E07351560803E07351760819E1CF
:105F7000000ED8809B559C6F010ED8A0E8069D6F3F
:105F80009CC3DEF3000160EC0BF080EC0BF097C3D8
:105F900000F098C301F099C302F09AC303F065D0F2
:105FA000030106D0030EDE6F000160EC0BF003016D
:105FB0000A0EDE6F000160EC0BF00301010E972763
:105FC000D8B0982BD8B4992BD8B49A2B740761D732
:105FD00006C183F307C184F308C185F301010951A8
:105FE0000F0B0301866F000180EC0BF003019A5147
:105FF0000101115D30E311E1030199510101105DCF
:106000002AE30BE10301985101010F5D24E305E14F
:106010000301975101010E5D1EE3030186510F0834
:10602000D8B002D0010117D0D8A441D68551FF08BD
:10603000D8B002D001010FD0D8A439D68451FF08BE
:10604000D8B002D0010107D0D8A431D68351EF08CF
:10605000D8B02DD6010100002D0E9EA8FED7AD6E42
:10606000006A016A026A036A000103C068F302C0A1
:1060700067F301C066F300C065F30301655307E1F0
:10608000665305E1675303E16853D8B4DFD0685322
:1060900007E1675305E1665303E16551040818E21F
:1060A000050E655D6D6F000E66596E6F000E6759C7
:1060B0006F6F000E6859706F746F6FC373F36EC3A8
:1060C00072F36DC371F3756B000140EC10F00301C6
:1060D000685307E1675305E1665303E1655103081F
:1060E00018E2040E655D6D6F000E66596E6F000E4E
:1060F00067596F6F000E6859706F746F6FC373F3D9
:106100006EC372F36DC371F3756B000140EC10F058
:106110000301685307E1675305E1665303E16551E5
:10612000020818E2030E655D6D6F000E66596E6F12
:10613000000E67596F6F000E6859706F746F6FC3F0
:1061400073F36EC372F36DC371F3756B000140ECB2
:1061500010F00301685307E1675305E1665303E15B
:106160006551010818E2020E655D6D6F000E6659FB
:106170006E6F000E67596F6F000E6859706F746F05
:106180006FC373F36EC372F36DC371F3756B00016C
:1061900040EC10F00301655306E1665304E16753D8
:1061A00002E1685318E0010E655D6D6F000E6659DF
:1061B0006E6F000E67596F6F000E6859706F746FC5
:1061C0006FC373F36EC372F36DC371F3756B00012C
:1061D00040EC10F0030168C374F367C373F366C344
:1061E00072F365C371F3010E756F000140EC10F09E
:1061F000D890036AF131026EF031016EEF31006E1A
:10620000EA2503016D6F01500001EB2103016E6F60
:1062100002500001EC2103016F6F03500001ED21DA
:106220000301706FEDC074F3ECC073F3EBC072F355
:10623000EAC071F3786F6FC377F36EC376F36DC303
:1062400075F3000124EC15F001C060F30001E0B724
:1062500001D0FDD7E09737D4DA510508D8A4DFD1B3
:1062600003016D6B6D5100014CEC02F003016D2BCD
:10627000006E00509EA8FED7AD6E160E6D5DF2E169
:106280000D0E9EA8FED7AD6E0A0E9EA8FED7AD6E6F
:1062900084B203D081A001D0FDD75E6B5D6B5C6BD7
:1062A0005B6B020E0001DE6FF2880301626B623DE0
:1062B00001D00AD02C0E6225E96E010EEA6ED8B02C
:1062C000EA2AEF6A622BF3D702012B6BEB0E2C6FDD
:1062D000170E01011B6F84B40FD00001DAEF1AF022
:1062E00003C0F5F002C0F4F001C0F3F000C0F2F01A
:1062F0000301648132D00101010E03016D6F0001C1
:1063000042EF1BF0F56BF46B02C0F3F001C0F2F04A
:106310000301636B5A51635D20E2D8906335026ECE
:10632000036A033602502D0FE96E020E0320EA6E57
:10633000ECCF6EF3ED52EFCF6DF30001F25103019C
:106340006D5D08E10001F35103016E5D03E16491AD
:1063500004D001D06481632BDDD764A14ED100014C
:10636000F55307E1F45305E1F35303E1F251040857
:106370001EE2050EF25D03016D6F000E0001F35980
:1063800003016E6F000E0001F45903016F6F000EE0
:106390000001F5590301706F746F6FC373F36EC31F
:1063A00072F36DC371F3756B000140EC10F0F5539F
:1063B00007E1F45305E1F35303E1F25103081EE250
:1063C000040EF25D03016D6F000E0001F35903012D
:1063D0006E6F000E0001F45903016F6F000E000193
:1063E000F5590301706F746F6FC373F36EC372F36B
:1063F0006DC371F3756B000140EC10F0F55307E1CC
:10640000F45305E1F35303E1F25102081EE2030ED7
:10641000F25D03016D6F000E0001F35903016E6F11
:10642000000E0001F45903016F6F000E0001F559D1
:106430000301706F746F6FC373F36EC372F36DC338
:1064400071F3756B000140EC10F0F55307E1F45364
:1064500005E1F35303E1F25101081EE2020EF25D81
:1064600003016D6F000E0001F35903016E6F000E02
:106470000001F45903016F6F000E0001F55903018B
:10648000706F746F6FC373F36EC372F36DC371F388
:10649000756B000140EC10F0F25306E1F35304E198
:1064A000F45302E1F5531EE0010EF25D03016D6F3E
:1064B000000E0001F35903016E6F000E0001F45944
:1064C00003016F6F000E0001F5590301706F746FC7
:1064D0006FC373F36EC372F36DC371F3756B000119
:1064E00040EC10F0F5C074F3F4C073F3F3C072F332
:1064F000F2C071F3010E0301756F000140EC10F062
:1065000001C061F30301612D3BD0D890036A000103
:10651000F131026EF031016EEF31006EEA250301B8
:106520006D6F01500001EB2103016E6F02500001FD
:10653000EC2103016F6F03500001ED210301706F27
:10654000EDC074F3ECC073F3EBC072F3EAC071F307
:10655000786F6FC377F36EC376F36DC375F3000185
:1065600024EC15F001C060F384B20BD0030160513C
:106570007308D8B402D0000104D081A001D0FDD7A7
:10658000000184A435D0020E03015A5D636F5A5195
:10659000635D29E2010E6325036A026ED89002361C
:1065A000033602502D0F016E020E032203C06FF35B
:1065B000D8906335026E036A033602502D0FE96EE0
:1065C000020E0320EA6EECCF03F0ED52EFCF70F332
:1065D0006FC3EAFF01C0E9FF03C0ECFFED5270C3D7
:1065E000EFFF6307D4D7F3C02EF2F2C02DF2000103
:1065F0003B0E9EA8FED7AD6E03015E530FE15D53C7
:106600000DE15C51FD080AE3D8B402D0010163D664
:106610005B51E608D8A002D001015DD63ED6030149
:106620006D6B6D51000165EC02F003016D2B006E86
:1066300000509EA8FED7AD6E0F0E6D5DF2E10D0EFF
:106640009EA8FED7AD6E0A0E9EA8FED7AD6E84B290
:1066500005D083A003D083A201D0FBD783B048D05C
:10666000780E626F62530DE0030EE16F00012EECB5
:1066700006F083A003D0030104D0000103016207E8
:10668000F1D783B035D0010EE16F00012EEC06F09A
:106690000301622B62511E082AE1626B010E0001A8
:1066A000F227D8B0F32BD8B4F42BD8B4F52B0101D2
:1066B00011510001F55D1AE314E1010110510001CF
:1066C000F45D14E30EE101010F510001F35D0EE3EF
:1066D00008E1F25101010E5DD8A002D0000106D000
:1066E0000001F56BF46BF36B010EF26F0301C9D778
:1066F00083B239D0780E626F62530DE0030EE16F02
:1067000000012EEC06F083A203D0030104D00001A7
:1067100003016207F1D783B226D0010EE16F0001B9
:106720002EEC06F00301622B62511E081BE1626B26
:10673000FF0E0001F227D8A0F327D8A0F427D8A095
:10674000F527F2530EE1F3530CE1F4530AE1F5534C
:1067500008E111C1F5F010C1F4F00FC1F3F00EC162
:10676000F2F00301D8D783A073D183A271D1626BF9
:10677000F5C074F3F4C073F3F3C072F3F2C071F3B5
:10678000756B000140EC10F001C061F30301615131
:1067900002080AE10001F56BF46BF36B010EF26F76
:1067A000730E0301606F15D1612D13D10001F553F4
:1067B00007E1F45305E1F35303E1F25104081EE24B
:1067C000050EF25D03016D6F000E0001F359030128
:1067D0006E6F000E0001F45903016F6F000E00018F
:1067E000F5590301706F746F6FC373F36EC372F367
:1067F0006DC371F3756B000140EC10F0F55307E1C8
:10680000F45305E1F35303E1F25103081EE2040ED1
:10681000F25D03016D6F000E0001F35903016E6F0D
:10682000000E0001F45903016F6F000E0001F559CD
:106830000301706F746F6FC373F36EC372F36DC334
:1068400071F3756B000140EC10F0F55307E1F45360
:1068500005E1F35303E1F25102081EE2030EF25D7B
:1068600003016D6F000E0001F35903016E6F000EFE
:106870000001F45903016F6F000E0001F559030187
:10688000706F746F6FC373F36EC372F36DC371F384
:10689000756B000140EC10F0F55307E1F45305E18E
:1068A000F35303E1F25101081EE2020EF25D03010F
:1068B0006D6F000E0001F35903016E6F000E0001B1
:1068C000F45903016F6F000E0001F5590301706F59
:1068D000746F6FC373F36EC372F36DC371F3756B33
:1068E000000140EC10F0F25306E1F35304E1F453DD
:1068F00002E1F5531EE0010EF25D03016D6F000E23
:106900000001F35903016E6F000E0001F4590301F9
:106910006F6F000E0001F5590301706F746F6FC344
:1069200073F36EC372F36DC371F3756B000140ECCA
:1069300010F0F5C074F3F4C073F3F3C072F3F2C057
:1069400071F3010E0301756F000140EC10F0D89057
:10695000036AF131026EF031016EEF31006EEA250B
:1069600003016D6F01500001EB2103016E6F0250B6
:106970000001EC2103016F6F03500001ED210301C1
:10698000706FEDC074F3ECC073F3EBC072F3EAC048
:1069900071F3786F6FC377F36EC376F36DC375F3DE
:1069A000000124EC15F001C060F384B213D00301A0
:1069B00060517308D8B402D000010CD083B003D06A
:1069C000730E606F06D083B203D0700E606F01D07B
:1069D000F5D70001030160516E0803E060517308B0
:1069E0000BE1010E0001F227D8B0F32BD8B4F42B41
:1069F000D8B4F52B2CD0030160517A080AE10001CC
:106A0000F56BF46BF36B010EF26F730E0301606FA5
:106A10001FD0605170081CE10001F55307E1F453E9
:106A200005E1F35303E1F251010809E2FF0EF227F9
:106A3000D8A0F327D8A0F427D8A0F52708D011C1F3
:106A4000F5F010C1F4F00FC1F3F00EC1F2F0030144
:046A500005D6030064
:067FF800A0F4C5FF00F13A
:00000001FF
